:100000000C9481040C94C8040C94C8040C94C80487
:100010000C94C8040C94C8040C94C8040C94C80430
:100020000C94C8040C94C8040C94562D0C94122DF6
:100030000C94562E0C94C8040C94C8040C94C80458
:100040000C94C8040C94C8040C94C8040C94C80400
:100050000C94C8040C94322E0C94C8040C94C8045C
:100060000C94C8040C94C8040C94C8040C94C804E0
:100070000C94C8040C94C8040C94C8040C94C804D0
:100080000C94C8040C94C8040C94C8040C94C804C0
:100090000C94C8040C94C8040C94C8040C94C804B0
:1000A0000C94C8040C94C8040C94C80405010902FB
:1000B000A10185020901A100050919012905150001
:1000C00025019505750181029501750381010501E1
:1000D000093009311581257F950275088106093897
:1000E0001581257F950175088106050C0A380215D2
:1000F00081257F950175088106C0C005010980A191
:1001000001850319012AB700150126B7009501756D
:10011000108100C0050C0901A101850419012AA064
:1001200002150126A002950175108100C005010984
:1001300006A1018505050719E029E71500250195A8
:1001400008750181020507190029EF1500250195A1
:10015000F0750181020508190129059505750191C0
:1001600002950175039101C00660FF0961A10109B3
:1001700062150026FF0095207508810209631500AD
:1001800026FF00952075089102C005010906A1010E
:10019000050719E029E71500250195087501810279
:1001A0009501750881010507190029FF150026FF33
:1001B0000095067508810005081901290595057542
:1001C000019102950175039101C00000000000003B
:1001D000000000000000000000000000000000001F
:1001E00000000000000000000000000000007E0F82
:1001F00000D4FFFFFFC700000078000000000000EF
:1002000000002A2B28000000000000000000000071
:10021000000000000029000000002C1E34202122D4
:1002200024342627252E362D3738271E1F2021223D
:10023000232425263333362E37381F0405060708B6
:10024000090A0B0C0D0E0F101112131415161718A6
:10025000191A1B1C1D2F3130232D350405060708E4
:10026000090A0B0C0D0E0F10111213141516171886
:10027000191A1B1C1D2F3130354C00047F3F1F64A1
:100280003214643214783C1E1E140A05FD377A5865
:100290005A000004E6D6B446020021011600000010
:1002A000742FE5A3E00359014D5D003D8889C654D4
:1002B00036C3174FE4DCC66B8B4E8235E020F54227
:1002C000FAECFA3EC64F2D6A8C88AD19EFC440B7E0
:1002D000D9EDF02C871F5E9FC901F5E0429165C101
:1002E0004C67FF4C49395D1D7746D96240A432AF57
:1002F000D7EC3FB6C15FE4B1EE60642DA920E7CB37
:10030000DAF5BF0CCAAF09448A4505B339718DCE01
:10031000361E2DB5E9B2108917741B2AD11A858BA8
:1003200079E038596B0A0D7A142FDF92B1089501E4
:100330004FB276A892C8E84BF3427196B746586C14
:100340004B3082EC727749F46FB565AC9DE127BF05
:10035000478044800B04A95A64CADA1DC343F9E1FB
:100360008F38FC2BCA7DF3BFA8E2D249DAF09A7825
:10037000608179927416C45C0AF2CA87FC700730F7
:100380000CCFE1DC72ABC78C8256E049A0228760BB
:1003900062B081B17C31694C6EA22CAC5D55E1F547
:1003A0009BED11ABDA57704AEA85B0773DB9291E4B
:1003B0007075B2EA018981582ECAC1D1BE62544912
:1003C000CC4D5F826F2DF9FB470FA659B0EBFC6F48
:1003D0001BDD9330619688B6C9552F4AEE08000C94
:1003E000BFAE7750E1EC1C012790B3EA4F391D7680
:1003F0002C905AA7739A920000000000ECF26482DD
:1004000028DB78960001E902DA060000B8E8BAC5F0
:10041000B1C467FB020000000004595A0001010149
:1004200001010101010102020202020202020203B1
:100430000303030303030304040404040404050581
:100440000505050606060606070707070708080844
:1004500008090909090A0A0A0B0B0B0C0C0C0D0DF3
:100460000D0E0E0E0F0F0F1010111111121213138B
:100470001414151516161717181819191A1A1B1B04
:100480001C1D1D1E1E1F2020212222232424252660
:1004900026272829292A2B2C2D2D2E2F3031323298
:1004A000333435363738393A3B3C3D3E3F404142A4
:1004B000434445464748494A4C4D4E4F505153548A
:1004C000555658595A5B5D5E5F616264656668693E
:1004D0006B6C6D6F7072737577787A7B7D7E8082BE
:1004E000838587888A8C8E8F91939596989A9C9E07
:1004F000A0A2A3A5A7A9ABADAFB1B3B5B7BABCBE17
:10050000C0C2C4C6C9CBCDCFD1D4D6D8DBDDDFE2E3
:10051000E4E7E9EBEEF0F3F5F8FAFDFFFFAA7F550B
:10052000402223252628292A2C2D2F3032333536F8
:10053000383A3B3D3E4042434547494A4C4E505174
:10054000535557595A5C5E6062646668696B6D6F9B
:1005500071737577797B7D7F81838587898A8C8E9E
:1005600090929496989A9C9E9FA1A3A5A7A8AAACA6
:10057000AEAFB1B3B4B6B8B9BBBCBEBFC1C2C3C5E0
:10058000C6C7C9CACBCCCDCED0D1D2D2D3D4D5D682
:10059000D7D7D8D9D9DADADBDBDBDCDCDCDCDCDDB5
:1005A000DDDDDDDCDCDCDCDCDBDBDBDADAD9D9D899
:1005B000D7D7D6D5D4D3D2D2D1D0CECDCCCBCAC931
:1005C000C7C6C5C3C2C1BFBEBCBBB9B8B6B4B3B160
:1005D000AFAEACAAA8A7A5A3A19F9E9C9A989694FB
:1005E00092908E8C8A89878583817F7D7B797775D0
:1005F00073716F6D6B6968666462605E5C5A5957AF
:10060000555351504E4C4A4947454342403E3D3B6D
:100610003A3836353332302F2D2C2A2928262523F7
:10062000222B0014001A00080015001700E000003B
:10063000001C0018000C00120013002A002C0000FF
:1006400000294104001600070009000A0002512891
:10065000000B000D000E000F0033003441E60003D4
:1006600053E1001D001B000600190005000000E317
:1006700000110010003600370038000251E500007C
:100680000035001E021F022002210222020100008A
:1006900000230224022502260227024C000100004A
:1006A000000100310034002D002E002F0001000158
:1006B0000030005100520050004F000100010000C6
:1006C0005C01002900C05C4600010001000000013F
:1006D000000100AD00AE00AC00AB00010001000065
:1006E0000035021E001F0020002100220001000032
:1006F000002300240025002600270001000100003F
:10070000002900310234022D022E022F02010001C5
:10071000003002210022002300A900010001000195
:1007200000010001000100010001000100000001C2
:100730000027001E001F002000AA00010001000089
:1007400000010001000100010001000100010000A2
:100750000001003A003B003C003D000100060000A3
:1007600000290001000100010001000100E2002C4D
:100770000001003E003F0040004100010001000177
:1007800000E1001E001F00200021002200000005E3
:100790000023004200430044004500010001000026
:1007A000000100010081040000020002007D04003D
:1007B0000003000100820400000400020067049BA3
:1007C0000705000100830400000600020069040020
:1007D00000070002007F04000008000100840400FC
:1007E00000090002006B0476070A0002006D04761F
:1007F000070B0002006F0476070C000200710476FC
:10080000070D000200730476070E000200750476DF
:10081000070F0002007704760710000200790476C3
:1008200007110002007B0476071200020085040015
:1008300000130002008704000009025B00030100AE
:10084000A032090400000103010100092111010087
:10085000012240000705810308000A090401000283
:100860000300000009211101000122220007058276
:100870000320000107050303200001090402000111
:100880000300000009211101000122BC00070584BA
:100890000320000A1201000200000008AEFE478893
:1008A0000100010203011C037600690061006C0075
:1008B0003A00660036003400630032006200330004
:1008C00063000000140343006100720061005600E1
:1008D00061006E0020003200000022035400680016
:1008E0006500560061006E0020004B006500790035
:1008F00062006F0061007200640073000000040376
:10090000090411241FBECFEFDAE0DEBFCDBF04B66D
:1009100003FE27C08091D7049091D804A091D904F8
:10092000B091DA048730904BA740B04BD1F41092CD
:10093000D7041092D8041092D9041092DA0414BE8D
:1009400084B7877F84BF0FB6F894A8958091600024
:10095000886180936000109260000FBEE0E0F8E3D1
:10096000099511E0A0E0B1E0EAE1FFE602C00590E0
:100970000D92AC3AB107D9F724E0ACEAB1E001C07E
:100980001D92A73DB207E1F70E94792E0C942537FE
:100990000C940000E8EDF0E080818E7F808310925F
:1009A000E2001092DA001092E100A0EEB0E08C912B
:1009B00081608C9380818F77808319BCA7EDB0E034
:1009C0008C918E7F8C9380818F7E808310929C048B
:1009D00008952091E4003091E50095E6A901209169
:1009E000EC00822F817020FF06C08091E80080FF1C
:1009F00006C080E008952091E80022FD1AC0809191
:100A0000CF04882389F0853089F08091EB0085FD43
:100A10000FC02091E4003091E50042175307F9F22E
:100A20009150E1F684E0089582E0089583E008950E
:100A300081E00895EF92FF920F931F93CF937C0173
:100A40008B010E94E904C82F811117C08091E80032
:100A500085FD0BC08091E8008E778093E8000E94AE
:100A6000E904882399F3C82F08C0F70181917F0119
:100A70008093F1000150110949F78C2FCF911F91FC
:100A80000F91FF90EF900895CF932091CF042430E1
:100A9000F9F4C091E900CF703091EC00232F217060
:100AA00030FD20E8C22B22E02093E9002091E800ED
:100AB00020FF0BC050E040E060E270E00E941A05A9
:100AC0008091E8008E778093E800CF70C093E900B2
:100AD000CF9108958091C70487FF13C08091E800EB
:100AE00082FF06C08091E8008B778093E80004C005
:100AF0008091CF048111F2CF08958091CF04882393
:100B0000D9F38091E80080FFF8CF8091E8008E77DC
:100B1000ECCF982F9093E900242F762F50E089177F
:100B200031F07091EC002091ED005091F00021FD2A
:100B300007C09F5F973071F78093E90081E00895C7
:100B40003091EB003E7F3093EB003091ED003D7F24
:100B50003093ED003091EB0031603093EB007093F7
:100B6000EC002093ED005093F0002091EE0027FD63
:100B7000E0CF80E00895CF92DF92EF92FF920F9343
:100B80001F93CF93DF93C8EDD0E088818F7E888359
:100B9000E7EDF0E080818160808384E082BF81E0C6
:100BA00080939C0488818E7F888302EE10E0F80198
:100BB00010821092DA0081EEC82ED12CF60110823C
:100BC00088818F77888388818068888388818F7DFA
:100BD000888319BC1092CF041092C6041092C504E9
:100BE0001092C40490EEE92EF12CF70180818B7FE6
:100BF000808388818160888342E060E080E00E9499
:100C00008905F60180818E7F8083F8018081816073
:100C10008083808188608083F70180818E7F8083DC
:100C2000888180618883DF91CF911F910F91FF9020
:100C3000EF90DF90CF900895FC01CB012091CD047F
:100C40003091CE042617370790F0009729F42091B1
:100C5000E8002E772093E80040E0009751F441111E
:100C600008C08091E80082FF31C080E00895C9018A
:100C7000F3CF2091CF042223A9F12530A9F12091AF
:100C8000E80023FD2DC02091E80022FDEACF20914D
:100C9000E80020FFE2CF3091F3002091F2000097AE
:100CA00019F02830310558F041E02830310509F0BD
:100CB00040E02091E8002E772093E800CECF4191CC
:100CC0004093F10001972F5F3F4FE9CF8091CF0410
:100CD000882341F0853041F08091E80083FFC1CF47
:100CE00081E0089582E0089583E008958091A3044F
:100CF00008959C014FB7F8948091930490919404C7
:100D0000A0919504B09196044FBF821B930B089558
:100D10002FB7F8948091930490919404A091950436
:100D2000B09196042FBF08959C01809125018823DE
:100D3000C9F08091970487FF15C0E62FE695E695E8
:100D4000E695603FE0F4E20FF32FF11D677081E05C
:100D500090E001C0880F6A95EAF780959281892317
:100D600082830895F9013296285F3F4F819168137D
:100D700003C0DF0111971C92E217F307B9F708953A
:100D80009C01809125018823C1F08091970487FF01
:100D900014C0E62FE695E695E695603FF8F4E20F7D
:100DA000F32FF11D677021E030E001C0220F6A953A
:100DB000EAF78281822B82830895F90132968FEFC0
:100DC00090E04191641751F08F3F19F4411101C037
:100DD000892F9F5F9630A9F78F3F09F40895280F58
:100DE000311D87FD3A95F9016283089520919104A0
:100DF000309192042817390771F0909392048093F0
:100E00009104E0918F04F0919004309721F00084D8
:100E1000F185E02D0994089520918D0430918E0480
:100E20002817390771F090938E0480938D04E09118
:100E30008F04F0919004309721F00680F781E02D27
:100E400009940895E0918F04F0919004309721F077
:100E50000190F081E02D099480E00895452B39F050
:100E6000682381E06F3F09F080E08170089581E0A0
:100E7000FCCFAC013091AF036091B003232F62131C
:100E800001C00895822F90E0FC01EE0FFF1FE9558D
:100E9000FC4F0190F081E02DE417F50791F467E035
:100EA000649FF001659FF00D1124E159FC4F41E072
:100EB00044832313E6CF0196837099278093AF0371
:100EC00008950196282F2370DACF10920C03109208
:100ED0000B03EFE6F3E08581811102C014821682D4
:100EE000379683E0E73AF807B1F70895E7E6F4E0CC
:100EF000848195812AE030E0B9010E940B3660932D
:100F00002001868180931F01828580931E01848544
:100F100080931D0186859785B9010E940B366093E9
:100F20001C01808980931B01828980931A01848926
:100F300080931901089580916704909168049093BB
:100F40002301809322010895FA0181110994FB0184
:100F5000FDCF089580919D04982F9E7F29F4817084
:100F6000826080939D0408958A34E8F381708864D8
:100F7000F8CF8F929F92AF92BF92CF92DF92EF9273
:100F8000FF920F931F93CF93DF93D82EC62EE901C4
:100F9000E42FF0E0E45EFB4F611113C04491942F05
:100FA000E42FE98348839A83DF91CF911F910F91BA
:100FB000FF90EF90DF90CF90BF90AF909F908F9079
:100FC0000895062F10E0E49186E0D89E7001112468
:100FD0002FEF30E0C701B9010E940B368D2D90E054
:100FE000880F991FF5E5F69FA001F79F500D11247A
:100FF000841B950B982F990F890FA901401B510B4A
:10100000E49FD001E59FB00D11244B2FC89E6001D5
:101010001124CD2CDD245901AC18BD08EA9D6001D6
:10102000EB9DD00C11249D2D4901881A9108809EBA
:101030005001819EB00C909EB00C1124AB2CBB24AF
:101040002A193B09E29F8001E39F100D11246330B0
:101050007105D1F08CEFE81683E0F80670F461308A
:101060007105B1F062307105B9F08FEFE816F10447
:1010700008F097CF9B2F412F94CF6430710579F002
:1010800066307105B9F38DCF4D2D9E2FEB2F89CF93
:101090004E2FED2D9B2F85CF912F4E2FF7CF9E2FCB
:1010A000E12F7FCF0E948806209155023091560291
:1010B000232B21F0809351029093520220915702EA
:1010C00030915802232B21F080934F0290935002CD
:1010D000E0918F04F0919004309749F082E0809382
:1010E00053020480F581E02D83E592E00994089590
:1010F00090915502803F59F48091560287FF0DC0B0
:101100001092560291110BC010924D0208C0813FFF
:1011100081F48091560218169CF3992381F08091F6
:10112000570290915802892B09F064C010924C022A
:101130000895823F49F497FFF0CF109255028091B5
:1011400056028111ECCFE0CF833F19F41916ACF3AE
:10115000E4CF20915702893F29F41216F4F6109239
:101160005702DBCF8A3F19F427FFD7CFF8CF209162
:1011700058028B3F29F427FFD0CF10925802CDCFD1
:101180008C3F19F41216CCF3C8CF843F31F4809110
:1011900054028E7F80935402C0CF853F21F480910A
:1011A00054028D7FF7CF863F21F4809154028B7FCC
:1011B000F1CF873F21F480915402877FEBCF883FA6
:1011C00021F4809154028F7EE5CF8D3F31F48091E0
:1011D0004E028E7F80934E02A0CF8E3F21F48091ED
:1011E0004E028D7FF7CF8F3F09F097CF80914E024F
:1011F0008B7FF0CF089580914E0280FF0CC06091EC
:101200001A0170E07595679575956795611571057B
:1012100049F1862F089581FF06C060911A0170E0A0
:1012200075956795F3CF60911A0182FD0BC090917F
:101230004C029923A1F06091190180911A0196172F
:1012400038F0682F70E06038710500F38FE708957B
:10125000899FC001112470E00E941F36F4CF61E025
:1012600070E0D7CF81E0089580914E0260916F04C5
:101270007091700480FF16C020911E01269FC0014E
:10128000279F900D1124BC017695679576956795FB
:101290006038710508F043C06115710509F441C05B
:1012A000862F089581FF0BC020911E01269FC0014B
:1012B000279F900D1124BC0176956795E9CF82FF99
:1012C00009C080911E019B01829FB001839F700D18
:1012D0001124DECF20914D022223D1F290911D01E5
:1012E00080911E01482F50E0291748F0CB01849FC0
:1012F000B001859F700D949F700D1124C9CF289F58
:1013000090011124269FA001279F500D369F500D5C
:101310001124692F70E0CA010E940B36B9CF8FE704
:10132000089581E00895803F31F40E943409819549
:10133000809356020895813F19F40E943409F8CF32
:10134000823F31F40E9434098195809355020895BB
:10135000833F19F40E943409F8CF893F29F40E9491
:10136000FB088093570208958A3F21F40E94FB08EE
:101370008195F7CF8B3F31F40E94FB0881958093D4
:10138000580208958C3F19F40E94FB08F8CF843F5F
:1013900031F4809154028160809354020895853F16
:1013A00021F4809154028260F7CF863F21F480912E
:1013B00054028460F1CF873F21F480915402886009
:1013C000EBCF883F21F4809154028061E5CF8D3FBF
:1013D00031F480914E02816080934E0208958E3FD9
:1013E00021F480914E028260F7CF8F3FB9F7809150
:1013F0004E028460F1CF80E008959091970492FFAF
:1014000006C0282F28712830F9F4877F846093FF65
:1014100006C0282F28712831F1F4877E846120913D
:10142000980420FF06C0382F38713830D9F4877FF0
:10143000816021FF06C0282F28712831D1F4877ED2
:10144000816194FD877E0895282F24712430F9F658
:101450008B7F8860DCCF282F2471243101F78B7EAD
:101460008861DDCF382F3171313019F78E7F886078
:10147000E0CF282F2171213121F78E7E8861E1CFC5
:10148000CF93DF93EC01803E910509F460C050F5E5
:101490008133910509F4A6C090F48932910509F4CD
:1014A0009AC08A9709F4A5C0C130D10509F462C079
:1014B000CE010497813A910508F055C05BC089338D
:1014C0009105F1F182389105D9F1C59709F47CC0F5
:1014D000C83AD10508F094C0C53AD10528F3A497BD
:1014E000D06448C0843E910509F453C068F4823E3C
:1014F0009105E1F1833E910509F440C0CE01805E83
:101500009109089780F536C0863E910509F44CC0D4
:10151000873E910509F44DC0811522E5920708F038
:10152000AAC0811531E5930708F0FAC08F3F9105F5
:1015300011F008F074C0803F910550F2D0651AC0D8
:10154000809197048370B1F0C0EED0E013C0809119
:10155000970480FD12C19091980490FF0BC0C3EED8
:10156000D0E084FF07C0D0E0C0E004C080919704C1
:1015700082FDF5CFCE01DF91CF9108958091970440
:1015800082FDFEC09091980490FDDECF84FFF2CFE3
:10159000EACF8091980481FFEDCF80919704C7EE48
:1015A000D0E084FDE0CFE6CF8091970483FDF7CFB4
:1015B000E1CF8091970483FDE6C09091980491FF5C
:1015C000E5CFC4EED0E0D6CF8091970485FFD2CF8F
:1015D000C9E2D0E0CFCF8091970485FFCBCFC5E3A0
:1015E000D0E0C8CF8091970486FFC4CFCAE2D0E094
:1015F000C1CF8091970486FFBDCFC1E3D0E0BACFC1
:10160000CF3BD10508F07ACFC85AD0E0CC0FDD1F10
:10161000CD5CDE4F0990D881C02DD464ABCF81154D
:1016200040E5940760F4C11580E4D80708F075C060
:10163000CE019A9581159F4108F49CCF94CFF4E098
:1016400096958795FA95E1F783702C2F2695269528
:10165000237040E2249F90011124382B8C2F83703B
:10166000C1E0D0E002C0CC0FDD1F8A95E2F7C22BAB
:10167000D32BDC687FCFC11586E5D80730F5C115BF
:1016800095E5D90708F060C0C11524E5D207C0F47C
:101690009C2F969596959E0123703327C115D345AF
:1016A00008F043C0C1E0D0E002C0CC0FDD1F2A9596
:1016B000E2F720E2929FC0011124C82BD92BD9CF89
:1016C000DC2FCC27C46FD06A55CFC1153AE5D307BC
:1016D00088F4C11549E5D40708F041C0CE019855FA
:1016E0008F3F910511F008F03ECFDC2FCC27C06F63
:1016F000D06A40CFCE0190568115904208F033CF8A
:101700008D2F8F710E94FD0990E0982F88278827E0
:101710009F719C012C2BE90120C0DF70D06A2ACF79
:10172000D82FCC27C16FD06A25CFC1E0D0E002C04E
:10173000CC0FDD1F2A95E2F730E2939FC001112400
:10174000C82BD92BDA6816CF8C2F0E94FD09C82F21
:10175000D0E0DC2FCC27CC27DF71D0620BCF8C2FD1
:101760008F700E94FD0934E0D695C7953A95E1F750
:10177000CF70DC2FC82FD069FDCEC9E3D0E0FACE00
:10178000C2EED0E0F7CEC6EED0E0F4CE80913402C7
:10179000882331F0109234021092330210923202F8
:1017A0000895982F9095809166048923809366040C
:1017B0000895982F909580916504892380936504FE
:1017C00008951092300210922F0210922E02089566
:1017D0008091690490916A04892B91F00E94880697
:1017E0002091320230913302AC01421B530B9A011B
:1017F00081E04091690450916A042417350708F488
:1018000080E0817008958091650490916604892B31
:1018100090913102892B8093AE018091340288230C
:1018200019F18091690490916A04892B29F00E9432
:10183000E80B81110E94C60B8091AE019091340299
:10184000892B8093AE0180912501882341F18091FD
:10185000970487FF24C08EE1E0EBF1E090E0815037
:1018600000F591110E94C60BE0918F04F091900455
:101870003097E1F080912501882359F080919704F9
:1018800087FF07C08091AE018093AF0185E0809310
:10189000AE010280F381E02D8EEA91E0099486E0AA
:1018A000DBCF21912223D9F29F5FD9CF0895CF9327
:1018B000DF93EC0181E0898B809165049F81892B06
:1018C00080936504809166049885892B80936604D3
:1018D0000E94030CEA81FB81309739F06C897D8985
:1018E000CE010696DF91CF910994DF91CF910895B3
:1018F000EF92FF920F931F93CF93DF93EC018A85B2
:10190000811134C0EB80FC8087E5F81A26E12E9D1A
:10191000C0012F9D900D1124DC01AB54BC4F1496D7
:10192000ED91FC911597309731F054966D917C9123
:1019300085549C4F099586E18E9D80018F9D100DE9
:1019400011240B541C4FF80187810E94D90BF80118
:1019500080850E94D10B0E94030C188219861B8679
:101960001E821D821092B4031092B303DF91CF91B7
:101970001F910F91FF90EF90089580912D0281119A
:1019800010922D020895E0912C029091EB01E91341
:1019900002C080E008952E2F30E058E0E59FF0016E
:1019A0001124E451FE4F5181561306C05081581343
:1019B00003C05281541304C0F9013196E770E7CF98
:1019C00081E0089580912C029091EB01981301C061
:1019D00008958F5F8770FACF9E3F41F1E92FE2951E
:1019E000E07FE80F982F9770E695E695E69583E0FF
:1019F000E89FF0011124EF52FE4F50E040E080E0FC
:101A0000219130E0092E02C0369527950A94E2F71D
:101A100021703327042E01C0220F0A94EAF7822B8B
:101A20004F5F5F4F4330510559F7089580E00895A7
:101A30009E3F59F1E92FE295E07FE80F877041E082
:101A400001C0440F8A95EAF7E695E695E69583E0AE
:101A5000E89FF0011124EF52FE4F30E020E070E0EB
:101A60005191DF011197CB01022E02C09695879507
:101A70000A94E2F7817081958527842385278C93CA
:101A80002F5F3F4F2330310559F70895282F892FB5
:101A900082958F70903C80F48A30B0F4843020F4CA
:101AA000823090F480E008958630E1F781E0283EAE
:101AB00088F0213FB9F70EC08C3011F08F3091F7CC
:101AC00093FB882780F9089581E0203F39F018F4CE
:101AD000283E40F70895243F29F7FCCF089590E071
:101AE00080E00E940C0790E080E00E94F6061092D1
:101AF0006604109231020E94030C86E0E3E5F2E0F6
:101B0000DF011D928A95E9F710924D0210924C0266
:101B100010924E020C9452088093D0040C946F0DD6
:101B20008091D004982F9670963019F488600C94A8
:101B30008C0D877FFCCF21E030E001C0220F8A9519
:101B4000EAF720958091D00482230C948C0D90911B
:101B500030028095892380933002282F277039F432
:101B6000282F082E000C330B9217130621F49091A6
:101B7000980492FF07C08595859585950E949B0DD9
:101B80000C94E10B089521E030E001C0220F8A950A
:101B9000EAF78091D004822B0C948C0D90919804DC
:101BA00092FD10C098E0899F90011124622B6093F0
:101BB00030020E94C30D0E94880690932F028093EA
:101BC0002E0208950C94C30D809335020C946F0D72
:101BD000882321F00E94D10B0C94030C08958823D4
:101BE00039F090916604892B809366040C94030C61
:101BF0000895882321F00E94D90B0C94030C0895BA
:101C0000882339F090916504892B809365040C94A6
:101C1000030C0895882379F19CEF980F913A38F4DA
:101C2000682F8EEA91E00E9494060C94030C90E2D7
:101C3000980F983050F4877091E001C0990F8A9501
:101C4000EAF7892F0E94D90BF0CF9BE5980F9330CC
:101C500020F490E080E00C940C0798E5980F973101
:101C600020F490E080E00C94F606803F20F00E9483
:101C700078080C9452080895CF93C82F882309F44C
:101C80006DC08CEF8C0F813AB8F5809125018823C7
:101C900011F18091970487FF1EC0EC2FE695E69521
:101CA000E695F0E0E255FE4F828190E04C2F4770C0
:101CB00021E030E002C0220F331F4A95E2F7822371
:101CC0009323892B89F06C2F8EEA91E00E94940671
:101CD0000E94030C09C0E0EBF1E08191C81799F371
:101CE00021E0E63BF207C9F76C2F8EEA91E00E94F3
:101CF000C006CF910C94030C80E28C0F883068F4FE
:101D0000C77021E030E001C0220FCA95EAF7809148
:101D10006504822B80936504ECCF8BE58C0F8330B8
:101D200038F42C2F2452330BC901CF910C940C079B
:101D3000E8E5EC0FE73150F4F0E0EE0FFF1FED5C4B
:101D4000FE4F80819181CF910C94F606C03F30F018
:101D50008C2F0E949309CF910C945208CF91089533
:101D60009C019A9581159F4150F5D901AA27B17020
:101D7000F901EE27F270B90166277470A9014427B2
:101D8000587034FF0EC080E1AB2B09F480E0EF2BDC
:101D900009F08062672B09F08064452B89F0806828
:101DA000089581E0AB2B09F480E0EF2B09F082600D
:101DB000672B09F08460452B19F08860089580E056
:101DC00008956F927F929F92AF92BF92CF92DF92CF
:101DD000EF92FF920F931F93CF93DF9329E9622E27
:101DE00021E0722E50E040E080E0C1E0D0E037ED2D
:101DF000C32E34E0D32E942EF301A1903F01B12CD9
:101E000005E911E070E060E0D8019D918D01E92FB6
:101E1000E295EF70F0E09F709E0101C0220F9A954D
:101E2000EAF77501062E02C0F594E7940A94E2F7EA
:101E300092A1E0FE55C0292B22A36F5F7F4F643033
:101E4000710511F7B0EABA95F1F78E0102C0000FE3
:101E5000111F9A94E2F75801A094B094E1EDF4E0D8
:101E600099EAE92E91E0F92E912C61917191D701B7
:101E70009D917D01292F22952F7030E0D9019096F8
:101E80002C9130E09F7002C0359527959A95E2F726
:101E900020FD29C09B01202B312B6217730741F0D5
:101EA000BF0162507109DB012D933C9399249394F7
:101EB000CE16DF06D1F689294F5F5F4F40315105BD
:101EC00009F099CFDF91CF911F910F91FF90EF9083
:101ED000DF90CF90BF90AF909F907F906F900895CC
:101EE00020952923A9CF9B012A213B21D6CF909170
:101EF000CF04943029F58093990460939A047093E9
:101F00009B049093E9008FEF9091E800815095FD3C
:101F100006C095ED9A95F1F700008111F5CF8091FB
:101F2000E80085FF0DC050E040E063E070E089E923
:101F300094E00E941A058091E8008E778093E80073
:101F40000895BC0184E00C94770FBC0183E00C94ED
:101F5000770F24E02093E9002FEF3091E800215023
:101F600035FD06C035ED3A95F1F700002111F5CFAA
:101F70002091E80025FF0BC050E040E066E070E0F3
:101F80000E941A058091E8008E778093E8000895FA
:101F9000CF93DF93D82FC92F809125018823C1F1DA
:101FA0008091970487FF34C060E284E08093E90069
:101FB0008FEF9091E800815095FD06C095ED9A95C0
:101FC000F1F700008111F5CF8091E80085FF1DC079
:101FD0008091250170E050E040E0811104C050E0A4
:101FE00040E068E070E08D2F9C2F0E941A058091E0
:101FF000E8008E778093E80080E2ED2FFC2FA4EAC2
:10200000B4E001900D928A95E1F7DF91CF910895A8
:1020100068E081E0CBCF81E08093E00080E28093B4
:10202000D8001092C9008FE19EE40197F1F700C03B
:10203000000087E090EBDC018093D7049093D804F4
:10204000A093D904B093DA0488E19CE00FB6F89429
:10205000A895809360000FBE90936000FFCF9C0115
:102060002150310908F408958FE99FE00197F1F7B5
:1020700000C00000F5CFFF920F931F93CF93DF9323
:102080008C01EB01F42E8091240182FF43C08B7FF1
:10209000809324018091890420918B0430918C04D9
:1020A000AB01421B530B9A01409122015091230135
:1020B00024173507A8F40E943C0E809124018D7FDF
:1020C0008093240180918504909186040E942F10B2
:1020D000809189040E940A0E82E00E94D10B24C0E4
:1020E000909166049260909366040E943C0E8091E9
:1020F00024018260809324018091820485FFE2CFD5
:1021000086FDE0CFFF20F1F2DF91CF911F910F917B
:10211000FF900895802F0E940A0E8091890490916B
:102120008A0480179107C1F20E94030CD0938C049B
:10213000C0938B04E9CF80919D0480FD0AC0E4E642
:10214000F2E0118210821282339652E0E03AF507F3
:10215000C1F7809A31B33E7F21B321604FB7F89425
:1021600084E692E0FC010196508168E021BB00000A
:1021700000C057FF31BB550F000000C000C000C0B9
:1021800031BB00C06A9591F752E0803A950751F74C
:102190004FBF8FE594E00197F1F700C0000008956C
:1021A000EF92FF920F931F93CF93DF93EC0104E61E
:1021B00012E0F12CE12C60919F0480919E049C819F
:1021C0002AE0E216F104FCF49923F9F09801409119
:1021D000A0040E94B9078FEFE81AF80A0D5F1F4F9D
:1021E00024E1E216F10439F70E949B108C8190E003
:1021F0000196817099278C83DF91CF911F910F9168
:10220000FF90EF900895992309F3980140E0E1CF02
:10221000CF92DF92EF92FF920F931F93CF93DF93B2
:10222000CDB7DEB72E970FB6F894DEBF0FBECDBF89
:102230008D879E87AD85BE8514961C91212F30E039
:10224000D9010E946A369B01AC010E9480366983E5
:102250007A838B839C83E0E2F0E0E11BF109A5E542
:10226000B0E09B01AC010E94803669877A878B873A
:102270009C879F01DF010E9462369B01AC010E9496
:102280008B366D837E838F8398879B01AC01898118
:102290009A81AB81BC81280F391F4A1F5B1F69855A
:1022A0007A858B859C850E943336F22E822F90E0B2
:1022B000A9E2A21708F442C0B3E02B9F90011124B9
:1022C00035952795122F109594E6C92E92E0D92EB8
:1022D00000E085E5E82EEF188E2D01FD8F2D96018B
:1022E000412F60919F040E94B9070F5FF3E0CF0E6A
:1022F000D11C043189F70E949B10AD85BE851496D0
:102300009C9181E0992319F0903219F48FEF80931A
:10231000180180911801890FED85FE8584832E9622
:102320000FB6F894DEBF0FBECDBFDF91CF911F91E6
:102330000F91FF90EF90DF90CF90089525E530E06A
:10234000F901E81BF90B9F01220F331F2E0F3F1FCE
:1023500037FFB6CF2F5F3F4FB3CF0F931F93CF936E
:10236000DF93C4E6D2E0FE0111821082128233961E
:1023700082E0E03AF807C1F710E000E080916202E5
:10238000082E000C990B081719078CF18091170182
:10239000082E000C990B801791074CF19E0140917B
:1023A000A00460919F0480919E040E94B9070F5F72
:1023B0001F4F23960431110509F70E949B1080914D
:1023C000160190916202980F90936202209117017A
:1023D000280F20931701121614F493311CF08195E5
:1023E00080931601DF91CF911F910F91089519826B
:1023F00018821A82DCCFCF92DF92EF92FF920F9376
:102400001F93CF93DF93FC018281DD24DA9480FD5A
:1024100002C0DD24D39404E612E0D0E0C0E0F8016D
:1024200011821082128294E0E92EF12CC12C80914D
:1024300061028C0D8531E4F164E10E94FD35892F44
:10244000082E000C990B8C179D0791F48091A00425
:102450008E9DA0018F9D500D112455954795559542
:102460004795980160919F0480919E040E94B9074E
:10247000CD0CF1E0EF1AF108D1F621960D5F1F4F58
:10248000C431D10561F60E949B108091610291E0F8
:10249000D91214C0811110C083E180936102DF91D1
:1024A000CF911F910F91FF90EF90DF90CF90089503
:1024B00087FFC6CF8C5EC4CF8150EFCF90E00196EE
:1024C000BE010E941F36E9CFEF92FF921F93CF9378
:1024D000DF93EC0184E6E82E82E0F82E10E08C8198
:1024E00097014091A00460919F04810F0E94B90759
:1024F000145F83E0E80EF11C103F89F70E949B10E7
:102500009A818C8190FF08C08F5F8C83DF91CF917F
:102510001F91FF90EF9008958150F7CF90919D0407
:1025200090FF0CC0E4E6F2E081836083428333963F
:1025300092E0E03AF907C1F70C949B1008950F93CD
:102540001F93CF93DF9300D00F92CDB7DEB78C01EE
:102550008091630281110AC09E012F5F3F4F4FEFB0
:102560006FEF0E94B9078A8180936302F80164814A
:10257000613049F06230F1F08091630240E06623FF
:1025800031F040E019C06091630240E080E00E94B9
:102590008E12F801848190E0019663E070E00E9461
:1025A0001F3684830F900F900F90DF91CF911F9172
:1025B0000F9108954091630280E060E0E8CFCF93EF
:1025C000DF9300D00F92CDB7DEB790919D0490FFBE
:1025D0000AC09E012F5F3F4F0E94B9074B8169815E
:1025E0008A810E948E120F900F900F90DF91CF91F1
:1025F0000895CF93DF93EC01EDE9F4E0438162812C
:102600008C810E94DF128C818F5F8C83DF91CF9150
:102610000895CF93DF93EC01EC81F0E0EF5DFA4F8A
:102620004491EDE9F4E0628181810E94DF128C81A6
:102630008F5F8C83DF91CF9108950F931F93CF937A
:10264000C82F0091870410918804893321F00091EC
:102650008504109186048C2F0E943C0E01151105F3
:1026600031F48C2FCF911F910F910C940A0E8FE9AA
:102670009FE00197F1F700C0000001501109EECF73
:10268000FF920F931F93CF93DF93C42FD22FFC01A0
:1026900082818823A9F040930A030E9488069093C0
:1026A000090380930803C77081E001C0880FCA95B1
:1026B000EAF7DF91CF911F910F91FF900C94000EDC
:1026C00010910A03141338C08091080390910903F4
:1026D0000E94790620917F0430918004821793072D
:1026E00058F5C0E2CD0F1D17A9F01770FF24F39421
:1026F0008F2D01C0880F1A95EAF70E94F90DC83096
:1027000048F48D2F877001C0FF0C8A95EAF78F2D52
:102710000E94000E802F0E941D13C830A0F4D770B5
:1027200081E001C0880FDA95EAF7DF91CF911F9120
:102730000F91FF900C94F90DC77081E001C0880FD4
:10274000CA95EAF7F2CFDF91CF911F910F91FF90D9
:102750000895AF92BF92CF92DF92EF92FF920F93C4
:102760001F93CF93DF93EC018AE0A82E28812223C8
:1027700009F48CC02130C9F599818A81913021F406
:1027800022960E941D1305C0923029F422960E94C1
:102790003C0E2196EBCF933021F422960E940A0E34
:1027A000F8CF943011F02196F4CF229630E020E05B
:1027B000AE014F5F5F4F8053990B8A30910550F007
:1027C0002150310930F38FE99FE00197F1F700C004
:1027D0000000F6CFA29EB001A39E700D11249C01B3
:1027E000260F371F8981EA01E3CFE22FF0E0E650A0
:1027F000FE4FB490822F86958695869590E0FC01D9
:10280000E651FE4FE4902770F12C022E02C0F594A1
:10281000E7940A94E2F731E0E322FF24FC01E65258
:10282000FE4FC490D12C022E02C0D594C7940A94B6
:10283000E2F731E0C322DD24FC01E653FE4F0491B0
:1028400010E002C0159507952A95E2F7017011274F
:10285000E114F10419F081EE0E943C0EC114D10480
:1028600019F086EE0E943C0E8B2D0E941D13CD2880
:1028700019F086EE0E940A0EEF2819F081EE0E94F0
:102880000A0E012B09F485CF8CE27BCFDF91CF912B
:102890001F910F91FF90EF90DF90CF90BF90AF907E
:1028A00008950F931F93CF93DF9307E614E0C7EAD1
:1028B000D1E0CE010E94D536F80181938F01219697
:1028C000C93CF1E0DF07A9F7C7EAD7E0FE0185912F
:1028D0009491009711F0FC0109952896F8E0CF3308
:1028E000DF07A1F7DF91CF911F910F9108950F930B
:1028F0001F93CF93DF93843038F5633028F5403150
:1029000018F520E2629FE0011124642F70E0660F49
:10291000771FC60FD71F30E6839FC00DD11D11242E
:10292000CE0187960E94D536082F10E0102F002781
:10293000CE0188960E94D5369801282BC901DF91D7
:10294000CF911F910F91089590E080E0F8CF462F2E
:10295000672F2091060330910703232B89F47E3FD4
:1029600039F44E3F69F48091040390910503089572
:10297000843030F4733020F4403110F40C94771428
:1029800090E080E00895DF92EF92FF920F931F9303
:10299000CF93DF937C010091D00480913502082B06
:1029A000C7E0D0E010E0DC2EC8010C2E02C09595E7
:1029B00087950A94E2F780FD0CC02197A0F7D12CEF
:1029C0008D2DDF91CF911F910F91FF90EF90DF90B0
:1029D0000895B7018C2F0E94A7140E94400A019706
:1029E00061F3EECFCF93DF93D82FC92F0E94C3148A
:1029F0006D2F7C2F0E94A714DF91CF910C94400A79
:102A0000FC0186819781009721F00E94400A0C9476
:102A1000460D808191810E94F214F9CF1F93CF93CC
:102A2000DF9300D000D00F92CDB7DEB749835A8331
:102A300089819A816623B9F02223A9F00E94C314E8
:102A4000182F682F89819A810E94180D69817A81D7
:102A5000812F0F900F900F900F900F90DF91CF91DB
:102A60001F910C94A7140E94EC0C182FEFCFFC01BF
:102A7000262F86819781009739F4408151816281A8
:102A8000738184810C940E15089583E290E00E9476
:102A9000D5368C3189F484E290E00E94D5368531B8
:102AA00059F485E290E00E94D53691E0873009F034
:102AB00090E0892F8170089580E0FCCFCF9384E06F
:102AC00090E00E94D536C82F82E290E00E94D53671
:102AD000982F8C2FCF9108950F931F93CF93DF934F
:102AE00007E614E0C7EAD1E0CE010E94D536F8012E
:102AF00061918F01681719F0CE010E94E936219685
:102B0000C93CF1E0DF0781F7DF91CF911F910F9171
:102B10000895E7E6F4E0128E138E8FEA90E0918339
:102B2000808385E0848F88E893E1938382834CE2FD
:102B300051E05583448322E330E03783268385E0E8
:102B400090E0918780878AE090E09387828764E1B4
:102B500070E0758764875787468744E650E0518B5D
:102B6000408B48E050E0538B428B48E250E0558B5D
:102B7000448B378B268B28EC30E0318F208F158EDD
:102B8000978F868F80E590E091A380A30E946C15BB
:102B90000C945114CF93DF93C9E6D2E060E0CE01EC
:102BA0000E94E9362196C11584E0D807B9F7DF9174
:102BB000CF9108950F931F93CF93DF9389018430B2
:102BC00050F5633040F5403130F521153C4531F486
:102BD0002091020330910303232BE9F090E2699FD7
:102BE000E0011124642F70E0660F771FC60FD71F16
:102BF00090E6899FC00DD11D1124612FCE018796CB
:102C00000E94E936602FCE018896DF91CF911F9107
:102C10000F910C94E936DF91CF911F910F91089598
:102C2000CF93C82F6FEF81116CE183E290E00E9497
:102C3000E9366FEFC11165E184E290E00E94E93668
:102C40006FEFC11167E085E290E0CF910C94E93617
:102C5000CF93C0919804C2FB992790F9981781F0FF
:102C600080FBC2F9C09398046091970484E090E0DF
:102C70000E94E9366C2F82E290E0CF910C94E93605
:102C8000CF9108957F928F929F92AF92BF92CF92F1
:102C9000DF92EF92FF920F931F93CF93DF93CDB705
:102CA000DEB764970FB6F894DEBF0FBECDBFA0901D
:102CB0000203B090030381E090E0909303038093BC
:102CC0000203912C812CE12C6401F12C15C0F80138
:102CD00025913491472D6F2D8E2D0E94DA150E5FB0
:102CE0001F4F739480E17812F2CFE0E1CE0ED11C39
:102CF000F394F3E0FF1639F08601000F111F0F5D0A
:102D0000194F712CE4CFE39480E3880E911CE4E02A
:102D1000EE12DACF0E9489151A8219821C821B8258
:102D20001E821D8218861F8288EC90E09A87898710
:102D300009EC11E04AE050E0B801CE0101960E9492
:102D40000D37065F1F4F0931F2E01F0799F77E012B
:102D50008BE0E80EF11C8AE0F70111928A95E9F701
:102D60004AE050E0B801C7010E940D37065F1F4FCF
:102D70000936F2E01F07A1F7B0920303A092020305
:102D800064960FB6F894DEBF0FBECDBFDF91CF9132
:102D90001F910F91FF90EF90DF90CF90BF90AF9079
:102DA0009F908F907F90089580E00E94101660E0C1
:102DB00086E290E00E94E9360E9442160E94CA15FF
:102DC00081E00C941016282FCB01283068F43AE0EB
:102DD000239FB001112467537E4F4AE050E00E94C8
:102DE000C53690E080E008958FEF9FEF08958F92B1
:102DF0009F92AF92BF92CF92DF92EF92FF920F938A
:102E00001F93CF93DF93CDB7DEB72A970FB6F89411
:102E1000DEBF0FBECDBF05EB13E0F12CE12C81E648
:102E2000C82E8CE2D82E9BE8A92E9CE2B92E2FEA60
:102E3000822E2BE2922EF801D182C082B382A2822E
:102E400095828482F58AE48ABE016F5F7F4F8E2D62
:102E50000E94E316892B29F489859A85F801938BC2
:102E6000828BFFEFEF1AFF0A0A5E1F4F88E0E81619
:102E7000F10409F72A960FB6F894DEBF0FBECDBF56
:102E8000DF91CF911F910F91FF90EF90DF90CF9046
:102E9000BF90AF909F908F900895CF92DF92EF9266
:102EA000FF920F931F93CF93DF93CDB7DEB72A978F
:102EB0000FB6F894DEBF0FBECDBFE2EBF2E080E5C7
:102EC000DF011D928A95E9F7EFE6F3E088E3DF0181
:102ED0001D928A95E9F782EBC82E82E0D82E7F01F9
:102EE00009E112E0F701D182C0824AE050E0B80166
:102EF000CE0101960E94C53688E0FE013196D601CA
:102F000001900D928A95E1F789859A85D7011396EC
:102F10009C938E931297BAE0CB0ED11CE7E0EE0E95
:102F2000F11C065F1F4F0936F2E01F07D9F62A96FB
:102F30000FB6F894DEBF0FBECDBFDF91CF911F91CA
:102F40000F91FF90EF90DF90CF900895109265045D
:102F500080912501E0EBF1E0882359F080919704FE
:102F600087FF07C08EE1DF011D928A95E9F70C9477
:102F70006F0D86E0F8CF1F93CF93DF93CDB7DEB709
:102F8000AA970FB6F894DEBF0FBECDBF87EC94E0D2
:102F9000FC0101962091F100208324E08F3C9207F0
:102FA000B9F78091C804893009F456C0C8F482305A
:102FB00009F4B2C0833009F481C0813071F180918D
:102FC000E80083FF35C18091C7049091C8049A300E
:102FD00008F02EC1E92FF0E0E95DF84C0C9455366D
:102FE0008A3009F488C08B3051F78091C704813250
:102FF00031F78091CB049091CC04892B01F780911B
:10300000E800877F8093E8000E946A058091C904E8
:10301000809325010E94A617D2CF8091C704813AE0
:1030200071F68091E800877F8093E8008091CB045F
:103030009091CC04892B61F460E284EA94E070E022
:103040000E941C068091E8008B778093E800B7CF40
:1030500060E090E080E0F3CF8091C704813209F016
:10306000AECF8091CB049091CC048D7F892B09F059
:10307000A6CF8091E800877F8093E8008091E800E8
:1030800082FF17C09091F3008091F200029729F41B
:103090008091F1008B7F813021F48091F100809349
:1030A000A3048091E8008B778093E8000E946A0572
:1030B00086CF8091CF048111E1CF81CF8091C70469
:1030C000813A09F07CCF8091CB049091CC04892B7C
:1030D00009F075CF8091E800877F8093E8008091A8
:1030E000E80080FFFCCF809125018093F100809162
:1030F000E8008E77D9CF8091C704813209F05FCF85
:103100008091E800877F8093E8000E946A058091A3
:10311000CA048093A20453CF8091C704813A09F076
:103120004ECF8091E800877F8093E8008091E8008F
:1031300080FFFCCF8091A204D8CF803899F08238EC
:1031400009F076C08091CB048F70873008F070C092
:103150008093E9008091EB0085FB882780F910922D
:10316000E90006C08091C4049091C5049111826069
:103170009091E800977F9093E8008093F10010927F
:10318000F1008091E8008E77C1C1882309F4AEC1B7
:10319000823009F04DC08091C9048111B2C1809183
:1031A000CB048F702FEF280F263008F041C080939A
:1031B000E9002091EB0020FFA4C1933031F480910D
:1031C000EB0080628093EB009CC19091EB009061DA
:1031D0009093EB0021E030E001C0220F8A95EAF7DE
:1031E0002093EA001092EA008091EB008860EACF19
:1031F00081111EC01091C9041F778091E30080786F
:10320000812B8093E3008091E800877F8093E80022
:103210000E946A058091E80080FFFCCF8091E30066
:1032200080688093E30082E0111183E08093CF04F3
:103230008091E80083FF0AC08091E800877F809337
:10324000E8008091EB0080628093EB00AA960FB6B5
:10325000F894DEBF0FBECDBFDF91CF911F910895CF
:103260008058823028F74091C9045091CA044C3DDF
:1032700083E05807A1F583E08A838AE289834FB708
:10328000F894DE01139620E03EE051E2E32FF0E0F7
:1032900050935700E49120FF03C0E295EF703F5F29
:1032A000EF708E2F90E0EA30C0F0C7968D939D931B
:1032B0002F5F243159F74FBF8091E800877F8093BB
:1032C000E8006AE270E0CE0101960E941C0680913F
:1032D000E8008B778093E800ABCFC096E7CF809172
:1032E000CB049091CC04252F33272330310509F4EA
:1032F0004AC078F52130310509F486C08BE590E0AD
:10330000E9E3F8E02230310509F092CF2091E8009E
:10331000277F2093E8002091CD043091CE048217BE
:10332000930708F49C0140E02115310509F071C0B4
:1033300041116FC08091E80082FDC9CF8091CF0418
:10334000882329F2853019F28091E80083FFF2CFBB
:10335000BECF2132310509F448C02232310509F0CF
:1033600067CF8330910508F063CFFC01EE0FFF1F9C
:10337000E757FE4F0190F081E02D8A579E4FDC0108
:103380008C9190E026C0CA019927423031F18330F8
:10339000910568F40097B1F0019709F049CFEAED83
:1033A000F8E0E4918E2F90E0EAEDF8E012C0039788
:1033B00009F03ECFE6EAF8E0E4918E2F90E0E6EAED
:1033C000F8E007C0EEEFF8E0E4918E2F90E0EEEF2A
:1033D000F8E0009709F42CCF99CFE4ECF8E0E49101
:1033E0008E2F90E0E4ECF8E0F4CF8330910508F004
:1033F0001FCF880F991FFC01E157FE4F0190F0810C
:10340000E02D89E090E082CF82E190E0E4E9F8E00D
:103410007DCF8091CF04882309F459CF853009F4FA
:1034200056CF8091E80083FD52CF8091E80082FD65
:1034300081CF8091E80080FF77CF9091F300809159
:10344000F2002115310519F08830910550F041E066
:10345000089709F040E08091E8008E778093E800BB
:1034600063CF44914093F100319621503109019688
:10347000E8CF803809F0DCCE8091E800877F809328
:10348000E8008091C6048093F1007BCE8111D0CEFC
:103490001091C904123008F0CBCE8091E800877FEC
:1034A0008093E8001093C6040E946A05112311F06E
:1034B00084E005C08091E30087FDFACF81E080932E
:1034C000CF0442E061EC81E00E94890542E261ECB8
:1034D00084E00E94890542E261EC82E00E94890555
:1034E00042E260EC83E00E948905A2CE8091C9048B
:1034F000813009F09DCE81E0933009F080E0809327
:10350000C5041092E9008091E800877F8093E8006D
:103510000E946A058DCE60919D04669570E04BE037
:1035200050E08BE091E00E94A836892B19F481E0ED
:10353000809360020E94880690935A0280935902F9
:1035400008950F931F93CF93DF938B01D82FC92F2B
:103550000E94AA07A8016D2F7C2F88E090E0DF91E0
:10356000CF911F910F910C94FB365F926F927F92D7
:103570008F929F92AF92BF92CF92DF92EF92FF9283
:103580000F931F93CF93DF9300D000D000D00F9202
:10359000CDB7DEB7182F762E042F622E90919D04A2
:1035A00090FF2BC0E92FE695AE2FB0E0AF59BE4F8C
:1035B0008C9180935F029E7F9230A9F59E012F5FD0
:1035C0003F4F812F0E94B9074B8169818A810E94F8
:1035D0008E1210939E0470929F040093A0046620A4
:1035E00061F080919D0490919E04A0919F04B09100
:1035F000A004BC01CD010E94A11A27960FB6F89431
:10360000DEBF0FBECDBFDF91CF911F910F91FF9015
:10361000EF90DF90CF90BF90AF909F908F907F9072
:103620006F905F900895823019F40091A004D1CF7B
:10363000863019F410919E04CCCF8930D9F38931AA
:1036400041F6E9518E2F8170582EE695F0E0E45E48
:10365000FA4FA590B490BB2484E6E82E82E0F82EC1
:10366000D12CC12C94E1892E912CC601B4010E9469
:103670000B36812F511013C0860F9701402F672DF5
:103680000E94B907CA0CDB1C93E0E90EF11CA0EA0A
:10369000EA16A2E0FA0649F70E949B109ACF861B11
:1036A000ECCFEDE9F4E0438121E1421B08F440E076
:1036B00021E0628181810C94B51AEDE9F4E0438147
:1036C00021E1420F08F44FEF21E0628181810C94E7
:1036D000B51AEDE9F4E0628121E1621B08F460E0D3
:1036E00021E0438181810C94B51AEDE9F4E0628117
:1036F00021E1620F08F46FEF21E0438181810C9496
:10370000B51AEDE9F4E0818121E0438162818850BE
:103710000C94B51AEDE9F4E0818121E043816281E6
:10372000885F0C94B51ACF93DF9300D000D0CDB74B
:10373000DEB78091A104882319F081508093A10401
:1037400080919D0490919E04A0919F04B091A0044B
:1037500089839A83AB83BC83BC01CD010F900F900A
:103760000F900F90DF91CF910C94A11ACF93DF931C
:1037700000D000D0CDB7DEB78091A104833018F41B
:103780008F5F8093A10480919D0490919E04A091ED
:103790009F04B091A00489839A83AB83BC83BC014E
:1037A000CD010F900F900F900F90DF91CF910C945F
:1037B000A11ACF93DF9300D000D0CDB7DEB79091A0
:1037C0009D0490FF42C09170811135C0926090932A
:1037D0009D04662381F080919D0490919E04A091A8
:1037E0009F04B091A00489839A83AB83BC83BC01FE
:1037F000CD010E94A11A60919D04669570E04BE096
:1038000050E08BE091E00E94A836892BD9F010920D
:10381000600281E080935C0220E04091A00460910E
:103820009F0480919E040F900F900F900F90DF9156
:10383000CF910C94B51A853210F09864C8CF880FD8
:10384000982BC5CF0E948B1AE4CF0F900F900F904A
:103850000F90DF91CF91089590919D0496958FEFF1
:10386000890F913009F484E261E00C94D91B8091B6
:103870009D0486958F5F853208F081E061E00C94AD
:10388000D91B90919D0490FF07C09695981720F042
:10389000961710F40C94371C61E00C94D91BCF934D
:1038A000DF9300D000D0CDB7DEB7EDE9F4E083E0E0
:1038B000808311828FEF8283838314828081918140
:1038C000A281B38189839A83AB83BC83BC01CD0180
:1038D0000F900F900F900F90DF91CF910C94A11A41
:1038E0006AEE7EEF90E080E00E94073760E082E0C1
:1038F00090E00E94E93660E083E090E00E94E936C3
:103900001092350260E084E090E00E94E93660E0C9
:1039100082E290E00E94E93660E085E090E00E945B
:10392000E93660E086E090E00E94E9366FEF87E0DC
:1039300090E00E94E93640E050E0BA0188E090E073
:103940000E94FB3660E08DE090E00E94E93640E0A6
:1039500050E0BA0188E190E00E94FB3660E087E128
:1039600090E00E94E93640E050E0BA018CE190E03E
:103970000E94FB3670E060E080E290E00E94073732
:1039800040E050E0BA0188E190E00E94FB3680E020
:103990000E9410160E94D41640E050E0BA018FE059
:1039A00090E00E94FB3640E050E0BA0183E190E0F5
:1039B0000C94FB368F929F92AF92BF92CF92DF9280
:1039C000EF92FF920F931F93CF93DF93CDB7DEB7A4
:1039D00028970FB6F894DEBF0FBECDBF7C01DC0187
:1039E00013964D915C91149711966C9111978C914F
:1039F0000E942E07811139C161E0C7010E9437156D
:103A00008C01F70182818111D2C0D70112964C91AD
:103A100041110FC10031BFE51B0709F4B9C10131E4
:103A2000EFE51E0709F4B8C1C80197558F3F91050E
:103A300011F008F04BC020910001022E000C330B56
:103A40002817390714F48093000126E1289F5001BC
:103A5000299FB00C112495012B543C4F6901D901C9
:103A600050964C935097F701928116968C91169729
:103A7000992309F493C11A961C930E9319978F5F9B
:103A800016968C930E948806D6011E969C938E9360
:103A90001D978091340217968C9317978091660436
:103AA00090916504892B18968C931897ED91FC9151
:103AB0001197309739F054966D917C91C5018554DA
:103AC0009C4F09951093B4030093B3038091820433
:103AD00080FFC3C10E9488066C01D70112968C91A9
:103AE000882311F18091240182FF06C040E0B601D5
:103AF00090E080E00E943B1082E00E94D10B0B31ED
:103B0000BCE51B0709F458C10C31ECE51E0709F4AC
:103B100089C190912401892F8E7F90FF81600A31A5
:103B2000FCE51F0709F481C10832110508F083C1C3
:103B30000E31110508F0AFC1C80104974A9708F08B
:103B400040C18091820484FD88C1D70112968C9176
:103B5000882309F4BCC18091240180FF7EC190912B
:103B6000820491FD04C020916504211176C195FF66
:103B70009DC120918B0430918C04F601E21BF30B64
:103B80009F0196FD02C081FD91C1283C310508F0DE
:103B90008DC12091890430918A040217130709F01E
:103BA00085C181FD7DC1802F0E943C0E53C0809154
:103BB00000018F3F09F429CF45EBC42E43E0D42EFA
:103BC000B12CA12C9924939480910001082E000C13
:103BD000990B8A159B050CF418CFF6018681882372
:103BE00009F1818592850817190739F48091B3038B
:103BF0009091B40308171907A9F0D6011F969C925B
:103C00001F971C961C930E931B9751968C918111B4
:103C100003C0C6010E94570CC60106960E94780C8C
:103C200010926604BFEFAB1ABB0AE6E1CE0ED11CC0
:103C3000CBCFC80182519F45409708F0BFC58FEF99
:103C400093E00E94D5363EEED32ED00E09E612E068
:103C5000882351F180913002877039F0F701828119
:103C6000882319F082E00E94A70D28960FB6F894D9
:103C7000DEBF0FBECDBFDF91CF911F910F91FF909F
:103C8000EF90DF90CF90BF90AF909F908F9008956E
:103C90000115F4E01F07F1F2C8010E94D536811129
:103CA00001C0DA940F5F1F4FD110F2CF809126012F
:103CB00090912701A0912801B091290189839A83CD
:103CC000AB83BC8399249A9468012FEFC21AD20A5D
:103CD000C8010E94D53689831A82882309F4BACF95
:103CE000813009F049C0580132E0A30EB11CC60171
:103CF0000E94D536C82E8A83882309F4ABCFC5012C
:103D00000E94D536D82E8FEF8C0D833068F4580181
:103D100043E0A40EB11CDB82DD2021F0CE01019630
:103D20000E94A9138501D0CF54E0C512FBCF5801E2
:103D300084E0A80EB11CC80103960E94D536282F36
:103D4000DD2009F487CF882309F484CF2150330B79
:103D5000929EA001939E500D1124AD2DA150BB0B3E
:103D6000CD01840F951F0197E8F2EFE9FFE031974D
:103D7000F1F700C00000F7CFCE0101960E94A91311
:103D80005601D0CF81E00E94C30D0E94900D62CFFA
:103D900081E00E949B0DF9CF82E0FBCF882309F4DC
:103DA00095CEF9018189882309F490CEC501855407
:103DB0009C4F0E94780C8ACE809124018160809370
:103DC0002401F7013281332309F404C510920A0358
:103DD0000631FCE51F0708F0B1C002302CE51207E0
:103DE00008F4B7C00E945E159093980480939704DE
:103DF00006313CE5130708F0D1C002304CE514074A
:103E000008F0BFC0609197041091980484E090E09E
:103E10000E94E936612F82E290E00E94E9360E941A
:103E2000A61718CF809124018E7F8093240182E011
:103E30000E94D10BC6CF0933110560F40D32110574
:103E400020F40B32110509F0BCCF8091820482FD71
:103E500004C07BCE04361105C1F3033FFCE51F0708
:103E600009F454C0D0F5083D3CE5130709F448C0F7
:103E7000093D4CE5140709F45BC0073D5CE51507F7
:103E800009F09FCF06E221EE41EE67ED7CE5C70128
:103E90000E944013DFCE8091820483FDDECF55CE99
:103EA000809166048260809366047DCE10938A04BC
:103EB00000938904D0928C04C0928B0480912401D9
:103EC00084608093240182E00E94A70DC3CE40E06D
:103ED000B601C8010E943B10BDCE053F8CE5180716
:103EE000D9F0063F9CE51907E9F0043FACE51A0755
:103EF00009F067CF07E225EE44EE64EF7CE5C7CF1B
:103F000007E225EE45EE68ED7CE5C1CF06E221EE45
:103F100040EE63EF7CE5BBCF06E221EE42EE65EFBB
:103F20007CE5B5CF07E225EE46EE66EF7CE5AFCF48
:103F300008E221E045EE69ED7CE5A9CFC8018A5F82
:103F40009C45099708F44ECF06314CE5140709F457
:103F500045C4809165048272063DFCE51F0708F0A8
:103F6000BDC0023C2CE5120708F4C4C0F801E35CB4
:103F7000FC45E331F10508F000C1EF5CF84C0C940E
:103F80005536F801E350FC45809197048160E33198
:103F9000F10590F4EC5BF84C0C9455360A5F1C4527
:103FA0000930110508F02ECF095A184CF8010C946D
:103FB00055368091970482608093970423CF809137
:103FC00097048460F9CF809197048860F5CF809141
:103FD000980481608093980415CF80919804826042
:103FE000F9CF809197048061E7CF80919704806238
:103FF000E3CF809197048064DFCF0E94A617809161
:1040000097048068D9CF809197048C60D5CF809138
:1040100098048360DFCF809197048E7FCDCF80910D
:1040200097048D7FC9CF809197048B7FC5CF8091F6
:104030009704877FC1CF809198048E7FCBCF8091EA
:1040400098048D7FC7CF809197048F7EB5CF8091E4
:1040500097048F7DB1CF809197048F7BADCF0E9465
:10406000A617809197048F77A7CF80919704837FBD
:10407000A3CF809198048C7FADCF8091970482FB71
:10408000992790F921E0922790FB82F990FB83F920
:1040900093CF80919804982F909591708E7F892B63
:1040A00090FB81F997CF0E94A61790919704892FD2
:1040B00097FB87F9805880CF61E08EE090E00E9406
:1040C000E936A0CE60E0F9CF8091CE0169E281119E
:1040D00065E38EEA91E00E949406ADC30D351007AA
:1040E00009F4B8CD81E00A35EDE51E0709F4D2C028
:1040F00008F0C1C001152CE5120709F4CEC00E3D31
:104100001C4509F4D7C0D70116968D919C91009754
:1041100009F4D5C00E94400A182F092FD701129622
:10412000CC9012971596DC90D2942FE0D2228091F9
:1041300030028770A1F0AC2CCC2091F0892F807FC9
:10414000803421F080E2810F883048F082E00E94C4
:10415000A70D809130028770AA24A3948111A12C0D
:10416000802F82958F70882E912C8C3008F0F3C0B0
:10417000F401E05AF84C0C94553680919D0480FF70
:1041800021C08E7F80939D0480919D0490919E0418
:10419000A0919F04B091A0048D839E83AF83B887C4
:1041A000BC01CD010E94A11A109260029FEFA0E70E
:1041B000B2E09150A040B040E1F700C000000E9482
:1041C0009B1048CD816080939D0461E086950E949C
:1041D000D91B40CD4CE25CE167E37CE10E94A4077F
:1041E00039CD47E35CE16CE27CE1F8CF41E85BE18B
:1041F0006AE87BE1F3CF4AE85BE161E87BE1EECF7F
:1042000049E65BE165E77BE1E9CF45E75BE169E62C
:104210007BE1E4CF41E55BE16DE57BE1DFCF4DE59F
:104220005BE161E57BE1DACF43E95BE166EB7BE1F2
:10423000D5CF46EB5BE163E97BE1D0CF61E081E084
:10424000C6CF65E082E00E94411C04CD68E086E0B4
:10425000FACF6EE089E0F7CF64E18FE0F4CF67E159
:1042600085E1F1CF61E088E1B2CF62E289E1EBCF95
:1042700061E083E2ACCF0B354DE51407F1F00C356E
:104280001D4509F040CF8091980482FB882780F972
:1042900091E089270E94281636CF0E94A6178FEF3B
:1042A00094E3ACE081509040A040E1F700C00000F2
:1042B0000E940B100E94701CCDCC80E0EBCFF70168
:1042C0008281C080D180882369F0C6010E94C31416
:1042D000182F682FC6010E94180DB601812F0E9469
:1042E000A71418CFC6010E94EC0C182FF6CFB02FE0
:1042F000BF70BB2E802F807F19F0B29490EFB9224F
:10430000CC20C9F0BB2069F080E2810F883010F02A
:1043100011110BC080916504B82AB09265040E9407
:10432000030C812F0E943C0E16C080916604B82AAF
:10433000B0926604F4CF812F0E940A0EBB2059F080
:1043400080E2810F883010F0111135C08B2D0E9452
:10435000D90B0E94030C98E0891A9108A4E08A16F0
:10436000910410F40E942207812F902F0E94460D85
:10437000811105C21092D0011092CF01AA20B1F094
:104380008091300280FD12C0D70112961C92859553
:10439000859585950E94C30DC7010E94DA1C809106
:1043A00030028595859585950E949B0D60E0C7013B
:1043B0000E9437155ACC8B2D0E94D10BCACFE02F0B
:1043C000EF70BE2E802F807F803219F0B29480EF84
:1043D000B822112321F1113009F46DC0CC2009F469
:1043E00076C0DD2009F446C020E0D7014C9111963B
:1043F0005C91119712966C91129713967C9113977A
:1044000014968C910E940E158091840481FD89CFB1
:10441000F701858180FF85CF8F7085832BC0CC20ED
:1044200069F1D11004C0809134028B2924C0F1E0DD
:10443000DF1213C08091980482FD8DCF80913402E9
:10444000B82AB81609F487CF0E94880690933302E1
:1044500080933202B09234027ECF80918304823006
:1044600010F3D812E0CF0E94C60B80912D02B81233
:10447000B0922D028B2D0E94000E6DCFD11006C080
:104480000E94C60B8B2D0E94F90D65CF809183048D
:1044900021E0D2120BC0823008F45DCF8091650418
:1044A0008B2109F458CF0E94BD0CEACF823040F333
:1044B000D812E6CF50CFCC2029F035E03D1508F4D6
:1044C0004ACFD8CF44E04D1508F445CFDBCFDD20EF
:1044D000C9F28091870490918804193321F080916A
:1044E0008504909186040E942F10812F0E940A0E4D
:1044F00032CF802F86958695837069F0813009F0E0
:104500002ACF812F902F9370C11002C090E080E0DD
:104510000E94F60620CF812F902F9370C11002C009
:1045200090E080E00E940C0716CF812FCC2039F05C
:104530000E9493090E9452080E9452080CCF0E94C8
:104540007808FACF802F837099F5C11004CF412FDE
:10455000429546954770440F440F812F8F70042E6B
:1045600001C0880F0A94EAF7212F207114FF07C0B9
:104570002FE030E001C0220F4A95EAF72095302F56
:10458000369536953370323071F0333051F04091BA
:104590003502313029F0822B84230E94E40DDBCEDA
:1045A000842B822BFACF282B809135028227F5CFDE
:1045B0008695CC2011F0802F8170882309F4CBCE12
:1045C000412F429546954770440F440F812F8F70BD
:1045D000042E01C0880F0A94EAF7212F207114FFDE
:1045E00007C02FE030E001C0220F4A95EAF720957E
:1045F000302F369536953370323071F0333051F0BC
:104600004091D004313029F0822B84230E948C0DFC
:10461000A2CE842B822BFACF282B8091D004822724
:10462000F5CFF02FFF70BF2ECC2029F08F2F0E94E6
:10463000C30D812F20CF812F0E94F90D8B2D0E9459
:104640009B0D89CE123F09F44AC060F4103F41F13E
:10465000113FE9F1CC2009F48DC0D11062CE802F3A
:104660008F713AC0133F09F43FC0143F99F720916E
:104670008304223008F466C080912D02CC2009F416
:104680004EC00E94D90B8091300287708430C1F5F2
:104690000E94E10B802F8F710E949B0DA12C5BCE9D
:1046A000CC2081F024E02D1508F455CE202F2F7159
:1046B00081E090E001C0880F2A95EAF79091D0043C
:1046C0008927A4CF35E03D1508F445CEEFCF802FE4
:1046D0008F71CC2009F4B3CF0E94C30D3CCE802F44
:1046E0008F71CC20C9F3ABCF80E0CC2009F48ECF02
:1046F00081E0902F9F7101C0880F9A95EAF786CFCD
:1047000080918304D81650F6402F4F71B42E842F19
:104710000E94C30D63E08B2D0E94CE0DBFCF909100
:104720006504982B90936504D21640F00E94E10B2B
:104730000E94BD0C64E0802F8F71EECF81E00E945B
:10474000A70DACCFCC2059F0502F5F71B52E852F1F
:104750000E94C30D63E08B2D0E94CE0DFCCD81E045
:104760000E94A70D81E08D1508F0F5CD82E00E9432
:10477000A70DF1CDD110ADCE802F8F7160CFCC20A1
:1047800019F0D110F7CDFACDD110F4CD20E0F7011A
:10479000408151816281738184810E940E158091D4
:1047A000840483FFE7CD8091CF019091D0010297DF
:1047B00009F0E0CD812F0E941D13DCCD0031FFE513
:1047C0001F0709F4DFCA01312FE5120709F02CC9D0
:1047D00082E0D9CA06311C4509F095CC8091650468
:1047E000982F9A7A2091810420FF04C0482F4474A6
:1047F00009F090E021FF04C0482F417109F090E0DA
:1048000022FF04C0482F487809F090E023FF03C03E
:10481000827209F090E0332309F456CC81E09111C3
:1048200001C080E08093CE0169E2911165E38EEAD8
:1048300091E00E94C0060E94030C0CCACF92DF9246
:10484000EF92FF920F931F93CF93DF938091E80134
:10485000807F31F48091E501C0912C0281110BC061
:10486000DF91CF911F910F91FF90EF90DF90CF904C
:1048700008952196C7708091EB018C1789F3F09011
:10488000E301E090E401C090E601D090E701A601C9
:104890006E2D8F2D0E942E07D0E08111EACF8E0160
:1048A00083E0000F111F8A95E1F7F801E451FE4FF4
:1048B00081818E11DECF80818F11DBCF82818111CA
:1048C000D8CFE380F480EC18FD0860E083EE91E03F
:1048D0000E94371580917F0490918004E816F906B4
:1048E00040F68091E8018F7080618093E801F801C3
:1048F000EF50FE4F80818F708061808383EE91E066
:104900000E94DA1CDF91CF911F910F91FF90EF90E1
:10491000DF90CF900C94E20C5F926F927F928F9217
:104920009F92AF92BF92CF92DF92EF92FF920F933E
:104930001F93CF93DF93CDB7DEB72D970FB6F894C3
:10494000DEBF0FBECDBF8C0185E0F801DE011996F8
:1049500001900D928A95E1F7D8011296EC9083EEC2
:10496000A82E81E0B82E8090E6019090E701A40186
:104970006091E4018091E3010E942E078111CEC174
:10498000F801C380D480F090E501C6018819990927
:104990004C01FF2009F45FC15080618060E0C501D7
:1049A0000E94371580917F04909180047090E801F7
:1049B0008816990608F020C14091E6015091E70160
:1049C000B090E301A090E401872D807F6A2D09F06B
:1049D000BAC08B2D0E942E07FE2C811139C0D80140
:1049E00011968C9111978A1133C08C918B1130C024
:1049F0002091E9013091EA0116968D919C9128173A
:104A0000390731F5E11024C0872D8F7080618093C4
:104A1000E80183EE91E00E94DA1C8091E801F80140
:104A200085838F2D2D960FB6F894DEBF0FBECDBFB8
:104A3000DF91CF911F910F91FF90EF90DF90CF907A
:104A4000BF90AF909F908F907F906F905F900895F0
:104A500060E083EE91E00E94371580917F04909191
:104A60008004843F9140F8F0A601662D852D0E94B8
:104A70002E0781114BC081E08E2580FF1DC04E2D79
:104A8000662D852D0E94C30C8823B1F083EE91E042
:104A90000E94DA1C88E0E3EEF1E0DF011D928A95C6
:104AA000E9F7F12CBECF60E083EE91E00E9437156C
:104AB0008091840480FDD8CFA601662D852D0E94AB
:104AC0002E07811125C081E08E25B82FB170DB2E15
:104AD00080FF30C04E2D662D852D0E94C30CC82E40
:104AE000811128C059866A8689859A850E94F214A8
:104AF000292F22952F70903268F0225F2F7022307C
:104B000088F0C8010E94DA1CCD2C12C080E0B5CF1D
:104B100080E0DBCF9F7011F0882351F0805E8830F9
:104B200038F0EFCF9F70D1F3F8019581907FB1F706
:104B3000FC2C77CFEE2009F474CF8091E8018160DE
:104B40008093E801AECF8B2D0E942E07811124C0E7
:104B5000D80111968C9111978A111EC08C918B11DE
:104B60001BC02091E9013091EA0116968D919C912C
:104B700017972817390781F4E1100EC015967C921B
:104B8000C8010E94DA1C88E0F801A3EEB1E00190B0
:104B90000D928A95E1F745CFC8010E940015882340
:104BA00039F1EE2029F18091E8018032A0F02091C6
:104BB000E3013091E4013A8329831B82DD82CC82B8
:104BC0008E838091E9019091EA0198878F83CE01CD
:104BD00001960E94DA1C88E0F801A3EEB1E0019092
:104BE0000D928A95E1F70E941E24FF24F39419CFB9
:104BF000C8010E94DA1CF9CF872D807F09F446CFC7
:104C00009090E3018090E4014091E6015091E7012A
:104C1000682D892D0E942E078111BECFF801818158
:104C20008811BACF80818911B7CF2091E9013091E5
:104C3000EA01868197812817390709F0ADCFE11085
:104C4000ABCF7582C8010E94DA1C88E0D5011D92A5
:104C50008A95E9F7E6CE60E083EE91E00E94371591
:104C600080917F04909180048816990608F050C0C6
:104C7000FE2CEE2009F4BCCFE090E301D090E401DB
:104C80004091E6015091E7016D2D8E2D0E942E0777
:104C9000811130C0F80181818D112CC080818E116D
:104CA00029C02091E9013091EA0186819781281776
:104CB000390701F560E083EE91E00E94371580919D
:104CC000840482FD60CF8091E80180FD5CCF982F45
:104CD000907F09F458CFD80115968C931597903F83
:104CE00009F44ECF982F907F905F8F70892B159687
:104CF0008C9346CFC8010E94001581116CCF809122
:104D0000E80181608093E801C8010E94DA1C89CE25
:104D100088E0F50111928A95E9F783CEEE2009F437
:104D200067CFC8010E940015F82E882309F460CFD0
:104D300088E0F801A3EEB1E001900D928A95E1F7C9
:104D40008091E3019091E4010E94F2140E941E24DC
:104D500068CEEF92FF920F931F93CF93DF93CDB75F
:104D6000DEB760970FB6F894DEBF0FBECDBF2987C0
:104D70003A874B875C876D877E878F87988BCE01BC
:104D800009960E948C24811136C088E0FE01399674
:104D9000DE01119601900D928A95E1F7E984FA847B
:104DA0000C851D85A8016F2D8E2D0E942E07811167
:104DB00022C0A091EB01B0E0CD0101968770992748
:104DC00020912C022817190649F1E982FA821D83E5
:104DD0000C8393E0AA0FBB1F9A95E1F7A451BE4F35
:104DE00098E0FE01319601900D929A95E1F780933B
:104DF000EB010E94E20C80912C029091EB0189134F
:104E00001BC060960FB6F894DEBF0FBECDBFDF911A
:104E1000CF911F910F91FF90EF9008950E94A617D8
:104E20001092EB0110922C0288E0E3EEF1E0DF013A
:104E30001D928A95E9F7DFCFB8E08B9FC00111245E
:104E400084519E4F0E948C248823D9F280912C0299
:104E500090E001968770992780932C02CCCFEF9237
:104E6000FF920F931F93CF93DF9380910E038823BC
:104E700061F0C0910D038CE0F82E80910E03C817ED
:104E800058F010920E0310920D03DF91CF911F91F5
:104E90000F91FF90EF900895EE24E394EC0EE092D2
:104EA0000D030C2F10E0CF9DE0011124C15FDC4FFA
:104EB0004B815C81698188810E942E0781111BC012
:104EC0008E819F81892B21F488859985019651F4E3
:104ED000288139814A815B816C817D818E819F81AE
:104EE0000E94A926F09EF001F19EF00D1124E15FD1
:104EF000FC4F14821382CE2DC0CF1092B2031092B9
:104F0000B103109221018091B0038093AF030E94FE
:104F100065070C942F273F924F925F926F927F927A
:104F20008F929F92AF92BF92CF92DF92EF92FF92B9
:104F30000F931F93CF93DF93C091AF0397E0892E18
:104F400001E010E02CE0322E3EEF932E44244394F7
:104F50008091B0038C1315C00E942F27DF91CF9151
:104F60001F910F91FF90EF90DF90CF90BF90AF9087
:104F70009F908F907F906F905F904F903F900C9498
:104F80006507D0E0FE01EE0FFF1FE955FC4F808161
:104F90009181889ED001899EB00D1124A159BC4FEA
:104FA00014962C911497211157C050900E03EFE0E6
:104FB000F3E030E020E0712C5D01251508F04AC0D7
:104FC000E284F384D501CD90DC906FEF7FEF612C0C
:104FD000462D50E0DA01AA0FBB1FAC0DBD1D0D9090
:104FE000BC91A02D109731F0EA16FB0609F4BA0126
:104FF0006394EECF6F3F7607A1F1D80102C0AA0FEC
:10500000BB1F6A95E2F77A2AB80102C0660F771FC4
:105010006A94E2F7AB014150510974161506F9F490
:10502000329EF001339EF00D1124E15FFC4F889E0B
:10503000D001899EB00D1124A159BC4F12962D911B
:105040003C91139737832683908291829187808742
:1050500015964C920E9439072196C37079CF14821D
:1050600013822F5F3F4F3C96A8CFCF92DF92FF92E3
:105070000F931F93CF93DF930E94E10E182F882385
:1050800061F181E0809338020E9488069093370294
:105090008093360280913602909137020E94790601
:1050A0000597F8F08091D1049091D2049093470233
:1050B000809346028091D3049091D4049093490246
:1050C000809348028091D5049091D60490934B022E
:1050D00080934A021092380204C0809138028111F4
:1050E000D9CF809100018F3F09F06AC080912101E2
:1050F00081116AC08091820480FF1CC080912401CC
:1051000082FF18C00E948806BC0180918B04909198
:105110008C049B01281B390B809122019091230163
:105120002817390738F041E08091890490918A046A
:105130000E943B10812FDF91CF911F910F91FF9023
:10514000DF90CF900895F29EF001F39EF00D1124B0
:10515000EB54FC4FC288D388C114D10421F4C09011
:105160007F04D0908004F29EE001F39ED00D1124C4
:10517000CB54DC4F8E818823B9F08D859E850E94AB
:105180007906C816D90680F40F9D6001112489891B
:10519000811105C0C6018B549C4F0E94570CC6015B
:1051A00085549C4F0E94780C0F5F202F30E0809137
:1051B0000001082E000C990B8217930724F696CF56
:1051C00000E086E1F82EF1CF8091B1039091B20317
:1051D000009709F48FCF0E94790620910B0330913C
:1051E0000C032817390708F085CF9091AF03809101
:1051F000B003981759F00E948B2710920C0310925D
:105200000B031092B2031092B10374CF0E942F27A8
:105210001092B2031092B1030E9465076BCF2F92D8
:105220003F924F925F926F927F928F929F92AF9236
:10523000BF92CF92DF92EF92FF920F931F93CF9383
:10524000DF93CDB7DEB769970FB6F894DEBF0FBE18
:10525000CDBF242F498B952F5A8B6B8B7C8B8D8BDD
:105260004C895D89692F822F0E942E07811109C008
:105270008091CF019091D00101969093D0018093BD
:10528000CF018B898111109266041E861F86188AB1
:1052900085E0FE017196DE01199601900D928A95C6
:1052A000E1F78091690490916A04892BC1F00E9412
:1052B000880620912E0230912F02821B930B2091A1
:1052C000690430916A048217930720F080913002BC
:1052D00082FFF2C10E94E80B81110E94C60B4C852F
:1052E0005D856A8589850E942E07811111C061E064
:1052F000CE0109960E9437156C018B8527EFC216E7
:105300002CE5D20681F4882321F181E080932101EC
:1053100029853A854B855C856D857E858F85988945
:105320000E94A926C5C038EFC3163CE5D30629F470
:10533000882379F00E947D27EBCF49EFC4164CE516
:10534000D40639F4882329F0809121018111F2CF0C
:10535000DCCF0FE613E0512CB12CA12C2224239496
:10536000312C2EEF422EF8014081518188248A94FD
:10537000982C20E0822F90E0FC01EE0FFF1FE40F3D
:10538000F51F608171816115710531F0C616D70670
:1053900009F44C012F5FEECFF12CFFEF8F169F0623
:1053A00009F448C0F8014481F09021018F2D41118A
:1053B00080E0F82FF170FF2EF801E58086819B8553
:1053C000992309F40CC1FF2009F409C160907D0400
:1053D00070907E04E11012C0A10101C0440F8A94B4
:1053E000EAF7842B868380910B0390910C0386153A
:1053F000970520F470920C0360920B03C10102C068
:10540000880F991F2A95E2F70197F801268128173E
:10541000190681F48091B1039091B203009709F4C9
:1054200060C00E9479066816790608F05AC021E02B
:10543000F80124835F28FFEFAF1ABF0A095F1F4FEF
:1054400028E0A216B10409F08ECF8B85882309F4D9
:105450001EC1552009F41BC10E9488069093B20317
:105460008093B10380910E03883010F591E0980F7E
:1054700090930E0398E0FE013996DE01119601909B
:105480000D929A95E1F73CE0839FC0011124815F62
:105490009C4F28E0FE013196DC0101900D922A9587
:1054A000E1F72FEF3FEFFC0131872087D386C286DB
:1054B00069960FB6F894DEBF0FBECDBFDF91CF91D6
:1054C0001F910F91FF90EF90DF90CF90BF90AF9022
:1054D0009F908F907F906F905F904F903F902F9014
:1054E00008958091AF035091B003982FF0E0E0E071
:1054F000851314C09093AF03E017F10709F49ACF16
:1055000090E0FC01EE0FFF1FE955FC4FB182A08235
:105510000196837099278093B0038CCF682E712CED
:10552000F301EE0FFF1FE955FC4F2081318147E069
:10553000429FD001439FB00D1124A159BC4F6D91E2
:105540007C911197798F688F40E020E030E0E32F65
:10555000F0E0EE0FFF1F688D798DE60FF71F80805A
:10556000918081149104E1F0F8010190F081E02D27
:10557000FF8BEE8B20E005C08616970609F44F2DB1
:105580002F5FE22FF0E0EE0FFF1F6E897F89E60F9D
:10559000F71F608171816115710571F73F5FD7CF8A
:1055A0004423D1F0F801231708F0FD0121E0248302
:1055B0000E171F0721F49093AF03F42E3BCF8913EE
:1055C00005C0AE17BF0711F49F5F937093012F5F63
:1055D0003F4F822F83708CCFF0E0E0E0F7CF90E078
:1055E000E1101FC0B10102C0660F771F2A95E2F7D4
:1055F0009B01215031092817390731F4442309F45C
:1056000044C0C5010E943907C10101C0880F8A94B6
:10561000EAF7982F9095F801868189238683FE2CDE
:1056200009CFAC01082C02C0559547950A94E2F7C2
:105630009C012150310982239323892B11F540FFCE
:1056400020C0F80182819381892BC1F01B821C82CA
:105650001D821E8249824A820E9488068160582FDC
:105660009D838C83F801828193818F839887298120
:105670003A814B816D817E810E94A926F8011582B5
:10568000C3CFF42FF170EF2EBFCFEF2CBDCF909191
:10569000AF038091B003981731F00E948B275520FB
:1056A00009F436CE05CF0E942F271092B203109234
:1056B000B1030E946507F3CF82E00E94A70D0ACED6
:1056C0000F931F93CF93DF9300D000D00F92CDB7ED
:1056D000DEB78C019093050380930403011580E2EB
:1056E000180720F5802F0E940A0EC8010E94B00EF4
:1056F0009801205E31092830310510F0012B59F452
:105700000F900F900F900F900F90DF91CF911F91FE
:105710000F910C94F90D0F900F900F900F900F9028
:10572000DF91CF911F910F910C94E80D8EEF89833B
:105730008A831B820E9488068160782F9D838C83D8
:1057400049815A816B818D810F900F900F900F903E
:105750000F90DF91CF911F910F910C940F290F9310
:105760001F93CF93DF938C01EB0168EA72E08C2FDB
:105770000E94E316892BA1F4809185049091860400
:105780000E942F10DD27C056DD4F8881F80110825E
:105790001882833009F148F4813059F0823081F069
:1057A000DF91CF911F910F9108958430D1F0853012
:1057B000B9F78091A8029091A902009789F306C0D9
:1057C0008091AA029091AB02009799F3DF91CF915B
:1057D0001F910F910C94602B8091AC029091AD02BF
:1057E000F3CF8091AE029091AF02009779F72091AC
:1057F000A8023091A9028091AA029091AB022115D2
:105800003105D9F2009711F7C901E0CF0F931F932B
:10581000CF93DF9300D000D00F92CDB7DEB78C01CD
:105820009093050380930403011580E21807E8F4C0
:10583000C8010E94B00E9801205E31092830310560
:1058400018F00115110571F40E94000E802F0F90C1
:105850000F900F900F900F90DF91CF911F910F91AC
:105860000C943C0E0E94EF0DF1CF8EEF89838A835A
:1058700081E08B830E9488068160782F9D838C83D2
:1058800049815A816B818D810F900F900F900F90FD
:105890000F90DF91CF911F910F910C940F29CF930F
:1058A000DF93D82FC92F0E94062C809185049091F8
:1058B00086040E942F108D2F9C2FDF91CF910C9486
:1058C000602B0F931F93CF93DF938C01862F68EA91
:1058D00072E00E94E316892BC9F4C091A802D0910E
:1058E000A902209799F0F8018081833069F4CE01F4
:1058F0000E944F2CCE010E944F2CCE01DF91CF9100
:105900001F910F910C944F2C8430B8F7DF91CF91F9
:105910001F910F9108950F931F93CF93DF938C01E5
:10592000EB0168EA72E08C2F0E94E316892B09F0E4
:1059300064C0FE01FF27D8018C91E056FD4F8130F5
:10594000D9F419969C911997992311F080830CC072
:105950001A969C919923D1F382E080838091AA02C8
:105960009091AB020097D9F48091A8029091A9027E
:10597000009709F442C013C08230E9F519968C9162
:10598000199781112DC01A968C9181110EC083E058
:1059900080838091AC029091AD02009719F1DF9164
:1059A000CF911F910F910C94062C84E080838091FD
:1059B000AE029091AF02009791F78091A80290916A
:1059C000A9020097F9F00E944F2C8091AA029091B1
:1059D000AB02009721F78091A8029091A902DFCF36
:1059E00085E080838091A8029091A902009729F018
:1059F0000E944F2CF0CF86E08083DF91CF911F91E2
:105A00000F9108958091AA029091AB02B1CF90E0DE
:105A100080E00E94E3368A3E9E4F11F40C944515B7
:105A200080E008951F920F920FB60F9211242F93CA
:105A30003F934F935F936F937F938F939F93AF9316
:105A4000BF93CF93DF93EF93FF93D091E900DF7083
:105A50008091EC00C82FC17080FDC0E81092E90071
:105A60008091F000877F8093F00078940E94BB17AC
:105A70001092E9008091F00088608093F000CD2BB7
:105A8000CF70C093E900FF91EF91DF91CF91BF916B
:105A9000AF919F918F917F916F915F914F913F91C6
:105AA0002F910F900FBE0F901F9018951F920F927D
:105AB0000FB60F9211242F933F934F935F936F93E1
:105AC0007F938F939F93AF93BF93EF93FF938091B7
:105AD000E10082FF09C08091E20082FF05C0809151
:105AE000E1008B7F8093E1008091DA0080FF24C089
:105AF0008091D80080FF20C08091DA008E7F809353
:105B0000DA008091D90080FF9FC080E189BD82E1E9
:105B100089BD09B400FEFDCF81E08093CF04809160
:105B20009C04811109C00E94CA040E94BB05809197
:105B3000E20084608093E2008091E10080FF17C062
:105B40008091E20080FF13C08091E2008E7F8093FD
:105B5000E2008091E20080618093E2008091D800B1
:105B600080628093D80019BC85E08093CF04809137
:105B7000E10084FF2DC08091E20084FF29C080E114
:105B800089BD82E189BD09B400FEFDCF8091D800B6
:105B90008F7D8093D8008091E1008F7E8093E1001B
:105BA0008091E2008F7E8093E2008091E20081602C
:105BB0008093E2008091C604882309F44BC084E0FE
:105BC0008093CF040E94A6170E9422070E948B1A7E
:105BD0008091E10083FF27C08091E20083FF23C012
:105BE0008091E100877F8093E10082E08093CF0481
:105BF0001092C6048091E1008E7F8093E100809135
:105C0000E2008E7F8093E2008091E20080618093C9
:105C1000E20042E060E080E00E9489058091F000AF
:105C200088608093F000FF91EF91BF91AF919F91B9
:105C30008F917F916F915F914F913F912F910F9035
:105C40000FBE0F901F90189519BC1092CF041092A0
:105C50009C0472CF8091E30087FD02C081E0B0CF49
:105C600083E0AECF78941F921FB61F9211248F93BA
:105C70009F93AF93BF938091930490919404A091CC
:105C80009504B09196040196A11DB11D80939304D3
:105C900090939404A0939504B0939604BF91AF9110
:105CA0009F918F911F901FBE1F9018951F921FB636
:105CB0001F9211248F939F93AF93BF93809193046E
:105CC00090919404A0919504B09196044196A11DE1
:105CD000B11D8093930490939404A0939504B09382
:105CE0009604BF91AF919F918F911F901FBE1F90FF
:105CF0001895CDB7DEB7E2970FB6F894DEBF0FBEAA
:105D0000CDBF84B7877F84BF0FB6F894A8958091E4
:105D10006000886180936000109260000FBE80E890
:105D200090E00FB6F89480936100909361000FBEED
:105D300085B7806885BF85B7806885BF8BEF99E0A0
:105D40009093AD018093AC010E94F7160E944D170D
:105D50000E9451140E94CA040E94BB058091E20077
:105D600084608093E20078948091CF048823A1F02E
:105D70001091E9001F709091EC00892F817090FDC7
:105D800080E8182B1092E9008091E80083FD0E94C2
:105D9000BB171F701093E90082E084BD93E095BDAE
:105DA0009AEF97BD80936E000E944515811102C045
:105DB0000E94D416A5E9B1E029E931E061E070E084
:105DC0008D91E82FE295EF70F0E091A18F70AB011B
:105DD00001C0440F8A95EAF7892F842B81A32A17E3
:105DE0003B0771F7A9EAB1E04CEA51E061E070E0ED
:105DF0008D91E82FE295EF70F0E011A18F709B017B
:105E000001C0220F8A95EAF7922F9095912391A3D2
:105E100082A1822B82A34A175B0751F71092D2040A
:105E20001092D10410924702109246021092D404AC
:105E30001092D30410924902109248021092D60494
:105E40001092D50410924B0210924A020E94072D24
:105E5000811102C00E94701C82E090E00E94D53641
:105E600080933B020E945E15909398048093970460
:105E70000E9435288FE39CE90197F1F700C00000EC
:105E80000E9435288091460280FF08C06FEF7FEFA7
:105E900090E080E00E9407370E940B1083E090E0C2
:105EA0000E94D5360E94E40D80913902811133C0E1
:105EB0000E94072D811104C00E94701C0E944F1C7B
:105EC00088E090E00E94DD3660939D0470939E040C
:105ED00080939F049093A0046E7F71F40E944F1CE6
:105EE00088E090E00E94DD3660939D0470939E04EC
:105EF00080939F049093A0040E94AA0710926002CE
:105F000080919D0480FF04C060E086950E94D91BAB
:105F100081E08093390281E091E090939004809336
:105F20008F045AE7252E52E0352EDE011396BCA7CA
:105F3000ABA7FE013D96FEA7EDA70E94352888235A
:105F400059F08FB7F8944091930450919404609164
:105F50009504709196048FBFA6E4B2E0ECE3F2E002
:105F600010E000E0702F8D919D91219131912817C3
:105F7000390709F4DCC02827392760E0EE24E394D0
:105F8000F12CA9014E215F21452B09F4CAC0698378
:105F90007A839C012E213F2191E0232B09F490E08C
:105FA0009B830E9488068160782F9D838C83498122
:105FB0005A816B818D810E940F29000F111FF801FA
:105FC000E45CFD4F80819181E826F926F182E08230
:105FD000809160028823D1F180915F02E0919D045D
:105FE000E695E81BE0935B02823009F0B7C0F0E071
:105FF000E857FD4FE4910E2F10E089E0E82E83E191
:10600000F82E80915C02882361F010925C020E945D
:10601000880690935A028093590210925E02109261
:106020005D020E948806E0915902F0915A028E1B8F
:106030009F0B8F3F9F4750F4E00FF11FF0935A02E0
:10604000E093590289E592E0F701099586E0E3E5DE
:10605000F2E0DE01119601900D928A95E1F7E09051
:106060005502F0905602009157021091580210927A
:1060700055021092560210925702109258028E2D1D
:106080008F2909F4CEC080915102909152020E9452
:1060900079069C0180914D02882309F4B8C0909143
:1060A0001F019217130608F0BCC08F3F19F08F5FD5
:1060B00080934D02EE2059F00E9434099FEF1E1488
:1060C0000CF491E0899F802D112480935502FF20CC
:1060D00059F00E9434099FEF1F140CF491E0899F3E
:1060E000802D11248093560230915502332309F4F8
:1060F00098C020915602222309F493C045EB340343
:10610000C0011124992309F4DCC09093550255EB8A
:10611000250390011124332309F4D7C0309356028C
:1061200080C06F5FEE0CFF1C603109F02ACF0F5F5B
:106130001F4F0330110509F015CF8FEF89A38AA3F4
:106140001BA20E9488068160782F9DA38CA349A181
:106150005AA16BA18DA10E940F293ACF863059F424
:10616000F0E0EB57FD4FE4910E2F10E0B9EFEB2E6E
:10617000B2E1FB2E46CF893061F4E695F0E0EE57B0
:10618000FD4FE4910E2F10E0A4E6EA2EA2E1FA2ED4
:1061900038CF8F3061F4E695F0E0E158FD4FE4919F
:1061A0000E2F10E0FBEFEF2EF1E1FF2E2ACF85310D
:1061B00059F4F0E0E458FD4FE4910E2F10E0EDEAC1
:1061C000EE2EE1E1FE2E1DCF08E210E058E0E52EB4
:1061D00051E1F52E883109F414CF833241F4F101F5
:1061E000059114917FE9E72E72E1F72E0ACF04EFB3
:1061F00011E060EDE62E60E1F62E843209F401CF65
:1062000000ED17E049EAE42E47E0F42EFACE409183
:106210002001FAE04F9FA00111244217530708F410
:1062200046CF812F802B09F45EC080914F02909160
:1062300050020E9479069C0180914C02882309F447
:1062400048C090911B019217130608F04CC08F3F75
:1062500019F08F5F80934C02002359F00E94FB08D5
:106260009FEF10160CF491E0899F802D11248093EC
:106270005702112359F00E94FB089FEF11160CF4EE
:1062800091E0899F802D112480935802309157020C
:10629000332349F120915802222329F145EB34039D
:1062A000C0011124992309F47CC09093570255EB47
:1062B000250390011124332309F477C03093580249
:1062C00012C081E08093550222CF81E08093560274
:1062D000A8CF40911C019AE0499FA00111244217C8
:1062E000530708F4B6CF8091550290915602892B3E
:1062F00090915702892B90915802892B11F00E949E
:106300005208EB82FC820D831E8386E0FE013196EB
:10631000A3E5B2E001900D928A95E1F70E94220771
:1063200090913A02891721F00E94220780933A0245
:106330008091CF04843009F000CE83E08093E9009F
:106340008091E80082FFF9CD8091E80090E085FF20
:1063500005C00E94E904882361F191E08091E80082
:106360008B778093E800992309F4E7CD0091060329
:1063700010910703E98101151105B9F1EE3F09F00C
:1063800069C08A81833020F08550833008F062C074
:10639000EA81EE3008F05EC0F0E0E459F84C0C946D
:1063A000553681E08093570282CF81E08093580276
:1063B0009ACF00E210E0CE0101967C018091E800C6
:1063C00085FD0AC08091E8008B778093E8000E94E9
:1063D000E904882399F3C1CF8091F100D7018D930F
:1063E0007D010150110951F7B8CFE43150F4EE238B
:1063F00051F0E150E33138F4F0E0E658F84C0C94F9
:106400005536EE3F29F28FEFCEC31A8289E08B8397
:1064100021C08A81823009F4E8C3833001F18130E0
:1064200091F78FB7F89420919304309194044091A0
:106430009504509196042FA738AB49AB5AAB8FBF48
:106440006FA578A989A99AA90E945B366B837C8382
:106450008D839E83CE0101960E9444056ECD80916E
:10646000020390910303892BA9F380914602909136
:1064700047029827892798279C838B83809148021D
:10648000909149029827892798279E838D83809130
:106490004A0290914B0298278927982798878F83E3
:1064A000D9CF8A81823009F0AECF8B819C81AD81BA
:1064B000BE818FA798ABA9ABBAABBC01CD010E943E
:1064C0005B3686E290E00E94E936C4CF4C816B8156
:1064D0008A810E9477149827892798279E838D8325
:1064E000B9CF2D813E813227232732274C816B8102
:1064F0008A810E94DA15AECF0E944216ABCF8A8104
:106500008238D1F1F8F4803831F1813809F0A2CF26
:1065100060E08B810E94D91B9B8180919D04911129
:1065200023C08E7F80939D04109260029FEFA0E7AE
:10653000B2E09150A040B040E1F700C000000E94DE
:106540009B1088CF833809F085CF20E04091A004CC
:106550006C818B8106C020E04B8160919F0480910B
:106560009E040E94B51A76CF816080939D0460E0FE
:1065700086950E94D91B6ECF8B818093A1046ACF30
:106580008A818238D9F058F4803899F0813809F03E
:1065900061CF80919D0480FF0FC0869538CF8338EE
:1065A00009F058CF80919E048B8380919F048C8347
:1065B00051CF8091A0042BCF80E029CF8091A104FE
:1065C00026CF20919D0430919E0440919F045091CC
:1065D000A0042FA738AB49AB5AABCA01B9010E943E
:1065E000A11A38CF80E18A8335CF81E08A8387E999
:1065F0000ECF8C81C82ED12C8D3108F02BCF0A8183
:106600001B81102701271027AE014F5F5F4F7A01D2
:10661000C40ED51EC80187599D4FEC14FD0409F422
:1066200019CF0739A1E01A0750F40E94D536F701B7
:1066300084830F5F1F4FBFEFEB1AFB0AEBCFD7012D
:1066400014961C92F6CF8091020390910303892B3C
:1066500009F400CF8C81C82ED12C8D3108F0FACEF0
:106660000A811B81102701271027FE0131967F0127
:10667000CE0EDF1EC80187599D4FEC14FD0409F4AE
:10668000E9CE073931E0130728F4D70114966C914D
:106690000E94E936BFEFEB1AFB0A0F5F1F4FEACFEC
:1066A0000E94CA15D7CE84E09ECF8C81C82ED12CF3
:1066B0008D3108F0CFCE0A811B81102701271027CA
:1066C000FE0131967F01CE0EDF1EC8018796CE14E3
:1066D000DF0409F4BFCE003831E0130758F40E94FC
:1066E000D536D70114968C930F5F1F4FFFEFEF1A2B
:1066F000FF0AEBCFF7011482F7CF8C81E82EF12C43
:106700008D3108F0A7CE0A811B81102701271027A1
:10671000003821E0120708F09DCE80E891E0801B50
:10672000910B8E159F0508F495CE480137E2830E34
:10673000911C80910203909103033701600E711E3A
:10674000892BC9F0AE014F5F5F4F7A01C801879670
:106750006016710609F47ECE003841E0140728F473
:10676000D70114966C910E94E936BFEFEB1AFB0A31
:106770000F5F1F4FEBCF680151E0C522DD2400FF02
:106780000DC0C80186960E94D5369D81892798271D
:10679000892781159C4511F48FEF8D83570160FE89
:1067A00017C0B1E0AB1AB10835E0432E512C4C0EA6
:1067B0005D1E4A0C5B1CC4018E0D9F1D0E94D536C8
:1067C000F201908181159C4519F48FEFD2018C93D1
:1067D000E1E0F0E0EC0FFD1FEC0DFD1D2FEFCA1402
:1067E000DB0408F0AFCF9481858181159C4511F4BD
:1067F0002483258332E0C30ED11C3296F0CF8091E2
:10680000020390910303892B09F424CECE01019653
:106810000E944405EFEFF1EE24E0E150F04020400B
:10682000E1F700C0000038CB88E0EAE2F1E0DE01E9
:10683000919601900D928A95E1F784E1ADA5BEA5F0
:106840001D928A95E9F784E089831A821B821C8253
:1068500088E0FE01B196DE01159601900D928A95B1
:10686000E1F7F8CD80E9898381E08A831B821C826D
:10687000F1CD8C81682F70E0762F66278B81860F93
:10688000972F911D092E000CAA0BBB0B25E0880F3A
:10689000991FAA1FBB1F2A95D1F7AC01BD01405E0D
:1068A0005F4F6F4F7F4F803EEFEF9E07AE07BE07F3
:1068B00008F0D0CD8039F1E09F07A105B10508F0BF
:1068C000C9CD413921E052076105710520F040E949
:1068D00051E060E070E0481B590BBC0164577D4FEC
:1068E000CE0101960E949F36B5CD4AE150E06FEF90
:1068F00070E0CE0107960E94BE3680910203898324
:106900000A831B821C8281E08D838DE08E83A2CD61
:1069100081E090E0909307038093060382E390E088
:1069200090934502809344020E948806909343020C
:10693000809342028FCD012B89F1F09046020091A5
:1069400048021091490280914202909143020E94B4
:1069500079068536910558F115FB002700F90023CB
:1069600031F1F0FE24C00E94880690934302809388
:106970004202809144029091450201979093450212
:1069800080934402892B51F410920703109206035E
:1069900081E090E0909303038093020380910203CF
:1069A0008983809106038A838091440230CD82E3FB
:1069B00090E09093450280934402F0CF109203033D
:1069C0001092020347CD0B811C8140E250E06FEF33
:1069D00070E0CE0101960E94BE3621EA37E090E0D9
:1069E00080E0AC014E5F5F4F4132510508F032CD7F
:1069F000F901659174910617170750F4A1E0B0E012
:106A0000AC0FBD1F8A0F9B1FFC0171836083CA01FD
:106A1000285F3F4FF8E029333F0719F71BCD2B8143
:106A20003C8181EA97E0FC01459154912417350798
:106A300009F4A3C0089648E089339407A1F7E3CC92
:106A40002B813C8101EA17E089E398E0F801459148
:106A500054912417350709F4A8C0085F1F4F801709
:106A60009107A1F7D0CC0E948915F4CC8B8182309C
:106A700009F447C058F481112DC08EE1ABA5BCA527
:106A80001D928A95E9F788E08983ADCD833009F4BA
:106A900056C0843009F0DECC6C818AE0FE01359668
:106AA000DE01919601900D928A95E1F78FEF6830A3
:106AB00068F4FAE06F9FB0011124675E7D4F4AE0F1
:106AC00050E0CE0181960E940D3780E089830E94BC
:106AD0004D17C0CC8C811AE07E01B1E2EB0EF11CA7
:106AE000F701212F11922A95E9F7B7010E94E316C9
:106AF0008983F701DE01129601900D921A95E1F754
:106B0000A9CC6C818AE0FE013596DE019196019058
:106B10000D928A95E1F78FEF683068F43AE0639F51
:106B2000B001112467537E4F4AE050E0CE018196B8
:106B30000E940D3780E089830E94F7168BCC6C8110
:106B40002AE0CE018196DC01E22F1D92EA95E9F759
:106B5000683088F4629FB0011124675E7D4F4AE07F
:106B600050E00E94C53680E089838AE0FE01B1963C
:106B7000DE01129672CE8FEFF7CF9C012E5F3F4F52
:106B8000F901459154914032510508F03CCCF9018E
:106B900045915491FC01349665917491CE01029611
:106BA0000E94B53680E0898355CCC8010296FC016D
:106BB000259134912D31310508F025CCFC0145910A
:106BC0005491F801349685919491BE016B5F7F4F8B
:106BD0000E94B5360E946C15F80136968591949105
:106BE000009701F3FC010995DDCF86E290E00E9459
:106BF000D5361B821C821D8289CE87FB082E062675
:106C000087FD819567FD61950E9493360EF49195FD
:106C100007FC81950895AA1BBB1B51E107C0AA1F61
:106C2000BB1FA617B70710F0A61BB70B881F991F2D
:106C30005A95A9F780959095BC01CD01089597FBD1
:106C4000072E16F4009407D077FD09D00E940B366A
:106C500007FC05D03EF4909581959F4F089570955F
:106C600061957F4F0895A1E21A2EAA1BBB1BFD015F
:106C70000DC0AA1FBB1FEE1FFF1FA217B307E4071B
:106C8000F50720F0A21BB30BE40BF50B661F771F73
:106C9000881F991F1A9469F7609570958095909553
:106CA0009B01AC01BD01CF010895EE0FFF1F0590C0
:106CB000F491E02D0994692796276927782787277B
:106CC000782708950E946A36332312F48A1B9B0B9F
:106CD0000C947B36A29FB001B39FC001A39F700D9F
:106CE000811D1124911DB29F700D811D1124911DD4
:106CF00008950E946A36B7FF0895821B930B08958A
:106D00000E946A36A59F900DB49F900DA49F800DA0
:106D1000911D11240895B7FF0C9480360E9480368F
:106D2000821B930B0895991B79E004C0991F961755
:106D300008F0961B881F7A95C9F780950895FB0186
:106D4000DC0102C005900D9241505040D8F70895E3
:106D5000FC014150504030F001900616D1F73197B8
:106D6000CF010895882799270895FB01DC0102C00F
:106D700001900D9241505040D8F70895DC0101C0B8
:106D80006D9341505040E0F70895DC01CB01FC01C8
:106D9000F999FECF06C0F2BDE1BDF89A319600B474
:106DA0000D9241505040B8F70895F999FECF92BD29
:106DB00081BDF89A992780B50895A6E1B0E044E036
:106DC00050E00C94C736A8E1B0E042E050E00C94EB
:106DD000C736262FF999FECF92BD81BDF89A01974B
:106DE00000B4021639F01FBA20BD0FB6F894FA9A13
:106DF000F99A0FBE08950396272F0E94EA360E9443
:106E0000E936252F0E94EA36242F0C94EA360196A3
:106E1000272F0E94EA360C94E936DC01CB0103C02F
:106E20002D910E94183741505040D0F70895262FD9
:106E3000F999FECF1FBA92BD81BD20BD0FB6F8945F
:106E4000FA9AF99A0FBE01960895F894FFCF9D180B
:106E5000C5181819C5181819F81830191819391A39
:106E6000461AEA20F120F620FB20002105210A2104
:106E70000F21142119211E212121262129212C2114
:106E80002F21322135213821D91FDF1FE31FF11FA8
:106E9000F51FF91FFD1F03200B200F2013201720C3
:106EA000232027202B202F20352053203D20E71F93
:106EB000ED1F1B201F200720392049205C20622065
:106EC00077217721DF21DF2179229522AB21AB21A8
:106ED000A2221123222322231434323439342A32B9
:106EE0002A32753488349B34DE34E3340F35203550
:106EF00033353635053209325132663271327C32E1
:106F00007F32C032E1320332FF33F232F532F932EE
:0A6F100023335033533355337D33E0
:106F1A00FF7606C80FA90FA50FA10F01191A1B1C8E
:106F2A001D1E1F2021220102012808641E140A3294
:106F3A001E01AF00010100000000EED2A737FC34A9
:106F4A003C8E00E200E900EA00B500B600B700CDC9
:106F5A00008301CC008A01920194012102230224B8
:106F6A00022502260227022A02B300B4006F00702B
:106F7A0000000102020202060606090909090909B6
:106F8A000F0F0F0F0F0F15151518191919191919B0
:106F9A001919191923244022BC8A016801AC004B33
:106FAA0008640884089496973401020304050600CD
:0C6FBA00070D0C0B0A090E0F08909192B5
:00000001FF
